:10000000CDC3000003C4000001C40000FFC3000012
:10001000FDC30000FBC30000F9C30000F7C30000EC
:10002000F5C30000F3C300000C9434310C941C326F
:100030000C94E930EBC30000E9C30000E7C3000003
:10004000E5C30000E3C30000E1C30000DFC300001C
:10005000DDC300000C941031D9C30000D7C30000E9
:10006000D5C30000D3C30000D1C30000CFC300003C
:10007000CDC30000CBC30000C9C30000C7C300004C
:10008000C5C30000C3C30000C1C30000BFC300005C
:10009000BDC30000BBC30000B9C30000B7C300006C
:1000A000B5C30000B3C30000B1C3000005010902DD
:1000B000A10185020901A1000509190129081500FE
:1000C0002501950875018102050109300931158165
:1000D000257F95027508810609381581257F9501D0
:1000E00075088106050C0A38021581257F95017572
:1000F000088106C0C005010980A101850319012AF4
:10010000B700150126B700950175108100C0050CD8
:100110000901A101850419012AA002150126A002E6
:10012000950175108100C00660FF0961A101096297
:10013000150026FF00952075088102096315002629
:10014000FF00952075089102C005010906A101056F
:100150000719E029E7150025019508750181029529
:1001600001750881010507190029FF150026FF0008
:100170009506750881000508190129051500250156
:10018000950575019102950175039101C00000006C
:10019000000000000000000000000000000000005F
:1001A000000000000000000000000000000000004F
:1001B000007E0F00D4FFFFFFC700000078000000A2
:1001C00000000000002A2B280000000000000000B2
:1001D000000000000000000029000000002C1E3478
:1001E00020212224342627252E362D3738271E1F7E
:1001F000202122232425263333362E37381F0405A9
:10020000060708090A0B0C0D0E0F10111213141516
:10021000161718191A1B1C1D2F3130232D350405F4
:10022000060708090A0B0C0D0E0F101112131415F6
:10023000161718191A1B1C1D2F3130354C09025B7B
:1002400000030100A0FA09040000010301010009F4
:100250002111010001224400070581030800010962
:100260000401000203000000092111010001222203
:100270000007058203200001070503032000010990
:100280000402000103000000092111010001227B8A
:10029000000705840320000112010002000000088D
:1002A000646975000200010203011C037600690005
:1002B00061006C003A0066003600340063003200D2
:1002C00062003300630000000A0349004400370065
:1002D000350000000E03490044004F004200410079
:1002E0004F0000000403090429001E001F00200025
:1002F000210022004C0023002400250026002700B6
:100300002D002E004600350014001A0008001500CC
:1003100017002A001C0018000C00120013002F0008
:10032000300039002B0004001600070009000A0005
:1003300028000B000D000E000F00330034003100C8
:100340004B00E1001D001B000600190005002800FD
:1003500011001000360037003800E50052004E0052
:10036000E0000405E300E20021522C002C002C00E8
:100370006152E600E4000F08500051004F00007C7D
:100380003A003B003C003D003E0000003F004000C2
:1003900041004200430044004500A500037CBD002D
:1003A00025782778237829782178D900D100CD00C5
:1003B000D200D9000000A600A700027CBE0026786B
:1003C000287824782A782278DA00CF00CE00D0006E
:1003D000DA00000000004A000100000000000000F8
:1003E0000000000020780000000000000000000075
:1003F000A800A9004D00010000000100010001005B
:10040000000000000000010001000100AE00AC008F
:10041000AA00AB0001000100010001000100010081
:1004200001000100010001000100010001000100C4
:1004300001000100010001000100010001000100B4
:1004400001000100010001000100010001000100A4
:100450000100010001000100010001000100010094
:100460000100010001000100010001000100010084
:100470000100010001000100010001000100010074
:100480000100010001000100010001000100010064
:100490000100010001000100010001000100010054
:1004A0000100010001000100010001000100010044
:1004B0000100010001000100010001000100010034
:1004C0000100010001000100010001000100010024
:1004D0000100010001000100010001000100010014
:1004E0000100010001000100010001000100010004
:1004F00001000100010001000100010001000100F4
:1005000001000100010001000100010001000100E3
:1005100001000100010001000100010001000100D3
:1005200001000100010001000100010001000100C3
:1005300001000100010001000100010001000100B3
:100540000001010101010101010102020202020296
:100550000202020303030303030303040404040469
:100560000404050505050506060606060707070730
:100570000708080808090909090A0A0A0B0B0B0CE5
:100580000C0C0D0D0D0E0E0E0F0F0F101011111182
:100590001212131314141515161617171818191903
:1005A0001A1A1B1B1C1D1D1E1E1F20202122222368
:1005B0002424252626272829292A2B2C2D2D2E2FA9
:1005C00030313232333435363738393A3B3C3D3EC0
:1005D0003F404142434445464748494A4C4D4E4FAF
:1005E00050515354555658595A5B5D5E5F61626471
:1005F000656668696B6C6D6F7072737577787A7BFE
:100600007D7E8082838587888A8C8E8F9193959654
:10061000989A9C9EA0A2A3A5A7A9ABADAFB1B3B574
:10062000B7BABCBEC0C2C4C6C9CBCDCFD1D4D6D850
:10063000DBDDDFE2E4E7E9EBEEF0F3F5F8FAFDFFEE
:10064000FD377A585A000004E6D6B446020021016C
:1006500016000000742FE5A3E0027500EA5D003D7E
:100660008889C65436C3174FE4E04BA1DB7A6EB4D9
:10067000D0C1E4A041996E0211E74DF2CD319855F9
:1006800023B102D8EBB4689F8FD885311D049C91AB
:10069000691A741F12190BBA49B1869D4527E934AE
:1006A0004742D123070D98CF7BA6F0DE687D94D119
:1006B00075E05998642031D0D94CC4BD513F418C6C
:1006C00079B37BF0A66294D5EA0A86931CEED637FE
:1006D00040F4280AD15063AD579988D730A591DCF2
:1006E000F213C087D9EE289D5CFDFE101D2F8EA849
:1006F00091AE71B7586C9A1E48E92E40DA9681E1A6
:100700003C0E317F14C672CFF425900EF097B6E2FE
:100710004540BE80394202627D47768D876F3AFD43
:10072000B0B2E19F7CE49B79A4B07D9DB79820791D
:10073000E8A7D7128CA76403FAEF47A5142702464F
:10074000F3F2D37E0FCBF5C2150000009E91A9A352
:100750001FB8FA1800018602F6040000DF9178D570
:10076000B1C467FB020000000004595A504F5251B7
:100770004A4D4B4E2A4C2F30B6B7ABACBBBCA9AAE6
:10078000BDBECFD0CDCEDBDCD9DA0D0E0B0F1A05F6
:1007900008050905071811130408120C11241FBEBF
:1007A000CFEFDAE0DEBFCDBF04B603FE18C0809104
:1007B000CE069091CF06A091D006B091D106873099
:1007C000904BA740B04B59F41092CE061092CF0632
:1007D0001092D0061092D106E0E0F8E3099526E0E9
:1007E000ACE0B3E001C01D92AE3CB207E1F713E00C
:1007F000A0E0B1E0EAE3F9E602C005900D92AC306A
:10080000B107D9F70E9473280C941B34F9CB9C01D3
:100810009A9581159F4118F5F32FF270EE27832FDB
:100820008170732F74706627532F5870442734FFDC
:100830000CC08295807FEF2B09F08062672B09F056
:100840008064452B69F080680895EF2B09F0826081
:10085000672B09F08460452B19F08860089580E0CB
:100860000895CF93DF93EB01D2DFFE010995DF916D
:10087000CF9108950C94CB320895982F92959F7044
:1008800024E0911102C020E0982F892F869586954B
:10089000811511F02E5F982F892F8695820F08956C
:1008A0008093CA0608958093CB06089521E030E036
:1008B00001C0220F8A95EAF78091CB06822BF3CFF5
:1008C00021E030E0A90102C0440F551F8A95E2F7EC
:1008D000CA0180959091CB068923E5CF292F9530C9
:1008E00090F58F3080F590E03FE0239F800D911DC3
:1008F0001124282F277041E001C0440F2A95EAF700
:1009000023E0969587952A95E1F7FC01EE0FFF1FEE
:10091000E80FF91FEA5CFA4F20E030E070E05191F7
:10092000DF01CB01022E02C0969587950A94E2F76B
:10093000817081958527842385278E932F5F3F4F74
:100940002330310561F70895292F953078F58F30E0
:1009500068F590E03FE0239F800D911D1124682FE2
:10096000677023E0969587952A95E1F7FC01EE0FD5
:10097000FF1FE80FF91FEA5CFA4F40E050E080E00B
:10098000219130E0062E02C0369527950A94E2F7B1
:1009900021703327042E01C0220F0A94EAF7822B1C
:1009A0004F5F5F4F4330510559F7089580E0089538
:1009B0009091CB0621E030E0F90101C0EE0F8A955D
:1009C000EAF7D90102C0AA0FBB1F6A95E2F7EA2B2A
:1009D00001C0220F4A95EAF7892F8E23E81303C03E
:1009E000892F822B60CF2095822F8923FBCF982FD0
:1009F00090958091CD0689238093CD060895803E01
:100A00009105D9F1C8F48133910509F482C048F405
:100A10008932910509F472C08A32910509F480C0C7
:100A2000089589339105E9F082389105D1F0853335
:100A3000910509F45EC00895843E9105D9F148F40A
:100A4000823E910539F1833E910549F181EE90E0B6
:100A50000895863E9105C9F1873E910509F43EC08F
:100A60000895209124052370211164C0209125054B
:100A700023FF14C089E290E008952091240520FD11
:100A800045C03091250530FF09C024FD24C083EE08
:100A900090E008952091240522FDF7CF089520913C
:100AA000240522FD44C03091250530FD43C024FFBC
:100AB000F5CF11C02091250521FFF0CF80912405AD
:100AC00084FD09C087EE90E008952091240523FF5E
:100AD000E5CF24FFF7CF80E090E008952091240532
:100AE00023FD2BC03091250531FFE1CF84EE90E04E
:100AF00008952091240525FFD1CFBCCF2091240556
:100B000025FD1EC02091250523FFC8CF89E390E075
:100B100008952091240526FFC1CF8AE290E0089530
:100B20002091240526FFBACF81E390E0089582EE5C
:100B300090E0089580EE90E0089586EE90E00895AC
:100B400085E390E008959091240592FF10C041E064
:100B5000282F2471243009F040E031E0282F28713B
:100B6000283009F030E0431711F02CE0822793FF82
:100B700010C041E0282F2471243109F040E031E019
:100B8000282F2871283109F030E0431711F02CE0AC
:100B900082273091250530FF10C051E0282F2171A8
:100BA000213009F050E041E0282F2871283009F069
:100BB00040E0541711F029E0822731FF10C041E0D6
:100BC000282F2171213109F040E031E0282F2871D0
:100BD000283109F030E0431711F029E0822794FD15
:100BE000877E08951F93CF93DF9309DFEC01811572
:100BF00020E59207D8F5811540E2940708F0E2C09D
:100C0000833C9105C0F4883A910508F098C0853A74
:100C1000910570F4049738F481E0219709F080E0A1
:100C2000C82F50E0D52FCE01DF91CF911F910895AD
:100C3000A497D064F8CF883E910558F4803E910582
:100C400090F78D5C9109D065439768F3C0E0D0E0E0
:100C5000EACF9A9581159F41C8F78D2F74DF182F21
:100C6000CE019927CCDEEC01D12BDDCFC03682E559
:100C7000D80738F5C03492E5D90708F07FC0C032F4
:100C800022E5D207B8F48C2FC11542E5D40708F04D
:100C900061C08F7158DF63E0CC0FDD1F6A95E1F70B
:100CA000CC27DF70282F30E084FD86C0C22BD32BE9
:100CB000D069B9CFCF71D0E0DC2FCC27C16FD06A1B
:100CC000B2CFC03C52E5D50708F5C03A62E5D60779
:100CD00008F06AC0CE0180569245809708F0B6CFE2
:100CE0008C2F86958695877050E2859FC0011124D0
:100CF000C37021E030E0A90102C0440F551FCA951E
:100D0000E2F7EA01C82BD92BDA688DCFCE01805CDF
:100D10009245809708F09ACFCE0123E0880F991F63
:100D20002A95E1F7807E9927C370DD2721E030E026
:100D3000A90102C0440F551FCA95E2F7E2CFC85A75
:100D4000D0E0CC0FDD1FC056DD4F0990D881C02DFB
:100D5000D46469CF8695869520E2829FC0011124D4
:100D6000C37021E030E0A90102C0440F551FCA95AD
:100D7000E2F7EA01C82BD92BDD6855CF8C2F869579
:100D80008695877050E2859FC0011124C37021E0D1
:100D900030E0A90102C0440F551FCA95E2F7EA01ED
:100DA000C82BD92BDC683FCF8C2F8F71CCDEC82F9E
:100DB000D0E0DC2FCC2737CF90E1899F9001112420
:100DC000332774CF99271BDEEC012DCF80E00895E7
:100DD000F894E82FE295EF70F0E041A18F7021E0E8
:100DE00030E0B90102C0660F771F8A95E2F7CB01A8
:100DF000962F9095942391A392A1892B82A3789406
:100E00000895CF92DF92EF92FF921F93CF93DF93DB
:100E1000172FE82FF0E0E05CFA4F71110CC0E4915D
:100E20008E2F7E2F6E2FDF91CF911F91FF90EF902D
:100E3000DF90CF900895E62EF12CC72ED12CF4919F
:100E4000EF2F86E0689F90011124CFEFD0E0C90119
:100E5000BE010E949E32AB01EE0CFF1C65E5649F53
:100E6000C001659F900D1124E81AF90A6E2D660FD6
:100E70006E0D7E01EC18FD08FE9DD001FF9DB00DAA
:100E800011248B2F169F70011124EF2CFF246E016B
:100E9000CE18DF087601FE9D6001FF9DD00C112465
:100EA0007E01E61AF108B701169F7001179FF00C3A
:100EB0001124EF2CFF24CE19DF09FC9F7001FD9F48
:100EC000F00C11247F2D43305105C1F02C3F3340ED
:100ED00058F441305105B1F04230510509F0A2CF2C
:100EE000EB2F8F2D7F2F9ECF4430510571F0463070
:100EF000510509F497CF7B2F8D2D94CF7D2DEB2FAE
:100F00008F2F90CF7F2FED2D8DCFEF2D7B2FF8CF13
:100F1000282F269F020E20E0211D1124822F0895E4
:100F20009C0180E090E0269F020E811D369F800D7F
:100F3000911D1124830F911D08959C01823091050C
:100F400008F408959FEF213E8EE1380740F4C9016F
:100F500045E0969587954A95E1F798E0980F61E00E
:100F6000E62FE90FFF27FF1FAF0155954795842F07
:100F7000449FF001459FF00DF00D11242E173F07FF
:100F800038F49FEF940F961758F78FEF860F089558
:100F90004F3FE9F361E0640FF6CFFC019B0100973E
:100FA00019F4832F80780895AC0197FF04C044277B
:100FB0005527481B590BB901640F751F37FD0FC02A
:100FC000C901841B950BA5E0880F991FAA95E1F72D
:100FD0000E94B23280E2861BF7FD81950895CB0115
:100FE00065E0880F991F6A95E1F7BA01621B730BE0
:100FF0000E94B23280E6EFCFCF93DF93D62FC72F78
:10100000682F2695E22F26FDE0959E2F9F7026FDE6
:101010009F5FE695E695E695E670F0E0EA5CFE4FA8
:101020003181399F302D912D112432953F70929549
:10103000907F392B8081830F27FD819587FD8195D6
:10104000880F66DF6D2F7C2FDF91CF9108950F936E
:101050001F93CF93DF93162FC72FD82F022FE42F84
:10106000F0E0EE0FFF1FE356FE4F64EE808150DF8D
:101070006C2F70E0482F50E0445E5F4F202F30E02F
:10108000CA01801B910997FF03C0C901841B950BFE
:1010900023E0880F991F2A95E1F79B01281B390B44
:1010A000C90137FF02C080E090E06C2F31DF782F5C
:1010B000612F8D2FDF91CF911F910F9108950F9385
:1010C0001F93CF93DF93162FD72FC82F022FE42F14
:1010D000F0E0EE0FFF1FE356FE4F64EE808118DF55
:1010E0006C2F70E0482F50E0445E5F4F202F30E0BF
:1010F000CA01801B910997FF03C0C901841B950B8E
:1011000023E0880F991F2A95E1F79B01281B390BD3
:10111000C90137FF02C080E090E06C2FF9DE612F3B
:101120007D2FDF91CF911F910F9108950F931F9302
:10113000CF93DF93162FC72FD82FBA01C9012C2FB9
:10114000201B022F2ADF982F990F990F891B6C2FD4
:10115000800FDEDE782F612F8D2FDF91CF911F91D1
:101160000F9108950F931F93CF93DF93162FD72FCF
:10117000C82FBA01C9012C2F201B022F0EDF982F78
:10118000990F990F891B6C2F800FC2DE612F7D2F65
:10119000DF91CF911F910F910895EF920F931F93BD
:1011A000CF93DF93162FC72FD82FBA01C9010E197D
:1011B0000C0FF3DE6C2F081B802FAADE782F612F17
:1011C0008D2FDF91CF911F910F91EF900895EF92A6
:1011D0000F931F93CF93DF93162FD72FC82FBA01EA
:1011E000C9010E190C0FD9DE6C2F081B802F90DE61
:1011F000612F7D2FDF91CF911F910F91EF90089577
:10120000622F0895E42FF0E0EE0FFF1FE356FE4F2C
:101210006081621B0895E42FF0E0EE0FFF1FE2569D
:10122000FE4F6081621B0895322F50E0FA01EE0FED
:10123000FF1FE256FE4F9081905297FD9195440F0B
:10124000551FFA01E356FE4F2081231B330B290F54
:10125000311D97FD3A95620F0895EF920F931F93FA
:1012600010E09801220F331F200F311F359527956D
:101270006E2D620F1F910F91EF9008950F93CF93F2
:10128000DF93D72FC82FB90147FD419528E330E000
:10129000241B310947FD3395229FA001239F500D48
:1012A000500D1124669FC001679F900D900D112471
:1012B000840F951F42DE982F990F692F680F600FDA
:1012C0007D2F8C2FDF91CF910F9108950F93CF93A6
:1012D000DF93D72FC82FBA01C9015FDE682F600FD7
:1012E0007D2F8C2FDF91CF910F910895CF93DF93B6
:1012F000D62FC72F682F842F80950ADE6D2F7C2F65
:10130000DF91CF9108951F93CF93DF93162FD72F9F
:10131000C82F60E4842F8095FBDD682F610F7D2F3F
:101320008C2FDF91CF911F910895EF92FF920F9331
:10133000970195E0099F200D311D1124211591E0A1
:10134000390710F02FEF30E02095382F320F08F4D6
:101350003FEF832F0F91FF90EF900895EF92FF9250
:101360000F93E00EF11CF90137FF03C0F195E195F1
:10137000F10924E0EE0FFF1F2A95E1F7E11531E0B6
:10138000F30714F0EFEFF0E09A0157FF03C0319537
:101390002195310994E0220F331F9A95E1F72E171A
:1013A0003F070CF4F901EE0DFF1DE11591E0F9077F
:1013B00010F0EFEFF0E02E2F2095382F320F08F4C9
:1013C0003FEF832F0F91FF90EF900895EF92FF92E0
:1013D0000F93972FFA01B9019701093430F4201BBC
:1013E0003109211541E0340710F02FEF30E0389635
:1013F000719740F0AB01485F5F4F4131510510F0EC
:101400002FEF30E02095382F320F08F43FEF832F75
:1014100077FF02C06D5F7F4F7595679575956795EE
:1014200020911005620F792F0F91FF90EF90089592
:10143000EF92FF920F939701201B3109211541E094
:10144000340710F02FEF30E0322F3095482F430F44
:1014500008F44FEF842F620F0F91FF90EF900895E3
:10146000EF92FF920F939701201B3109211591E014
:10147000390710F02FEF30E02095382F320F08F4A5
:101480003FEF832F0F91FF90EF90089590915304B9
:10149000982B90935304089526C108952FC1089561
:1014A00091E1899F802D1124980F963508F095E5DC
:1014B0000895EFE0F5E0808191E089278083109224
:1014C000090181E0E3CF80910F058370811102C093
:1014D0001092090180910F058C7F816080930F0528
:1014E000089580910F0583708111109209018091F8
:1014F0000F058C7F80930F050895982F862F2091DC
:101500000F052370211581F0911579F0913278F44F
:101510009F73990F990F20910F052370922B909331
:101520000F0510920901B2CF089591E0F2CF90E239
:10153000F0CF80910F05869586958F5F813208F0F8
:1015400081E061E0DACF80910F05869586958A95D6
:1015500009F480E261E0D1CF982F822F20910F050E
:101560002370211539F09093100560931105409375
:1015700012058CCF0895EFE0F5E0818190E021E045
:10158000438162810896E8CFEFE0F5E0818121E0B8
:10159000438162818850990BDFCFEFE0F5E06281F3
:1015A00020E1620F08F46FEF818121E0438190E038
:1015B000D3CFEFE0F5E0628120E1621B08F460E048
:1015C000818121E0438190E0C7CFEFE0F5E04381E6
:1015D00020E1420F08F44FEF818121E0628190E029
:1015E000BBCFEFE0F5E0438120E1421B08F440E08F
:1015F000818121E0628190E0AFCFEFE0F5E02481CE
:1016000030E1230F08F42FEF248381E03FCFEFE098
:10161000F5E0248130E1231B08F420E0248381E0FD
:1016200035CF81152CE7920741F4209121053091A7
:101630002205232B11F480E090E00895EDE4F6E01C
:1016400080E090E061E977E244EB57E226E238E29D
:10165000768365835087478332872187968785877E
:1016600001963F968830910599F70895FB01811501
:1016700020E2920728F4811541E0940738F4089598
:101680009C0130522115304348F00895392F94FFC2
:1016900002C03295307F2081232B20839927089523
:1016A000462B22FF0FC0982F92959F708F70892B29
:1016B000962F92959F706F70692B942F92959F70C3
:1016C0004F70492B982F9623961309C050E04095F0
:1016D000509590E04823592381E0452B09F080E0A4
:1016E0000895809A0895FC01EE0FFF1FE80FF91F7F
:1016F000EC5CFC4F6183408322830895FF920F933B
:101700001F93CF93DF93182F062FF42EC0E0D0E065
:101710002F2D402F612FCE01E6DF2196C535D10553
:10172000B9F7CDB7DEB7E5E00C949032FC018481C7
:10173000862381110AC082818115B9F068239085C2
:1017400093FF05C081E061110FC080E00895282F4C
:1017500022952F708F70282B962F92959F706F7007
:10176000962B81E02913F1CF089581E008950F931E
:101770001F93CF9301E010E0082E01C0000F0A94E0
:10178000EAF7C091C9069C2F9023911108C08ED80A
:10179000C027C093C906CF911F910F91089590D88B
:1017A000F7CF282F35EB2303C001112497FF04C086
:1017B00080589109892F089580589F4FFBCF8091C1
:1017C000560580FD14C081FD14C082FD16C08091B5
:1017D0005505811581F08E3180F420E5829FC0018E
:1017E00011246EE170E00E94B232862F089584E1E8
:1017F000089588E2089588E0089580E5089580912D
:10180000560580FD17C081FD17C082FD19C080916B
:101810005405811599F0883298F428E0829FC00120
:10182000112468E270E00E94B2326115710551F036
:10183000862F089562E0FCCF64E0FACF61E0F8CF34
:1018400068E0F6CF81E008959091B005890290019B
:10185000112437FF03C08093B00508952F37310559
:101860001CF4980F9093B00508959C0180E090E0DF
:10187000F901E80FF91FE491E41307C091E089270B
:10188000F901E80FF11D849108950196861780F300
:1018900080E00895FA01309709F009950895E091E4
:1018A0002C05F0912D05309739F00190F081E02D55
:1018B000309711F00995089580E00895A3E0B0E015
:1018C000E4E6FCE00C9477329C0180913203909125
:1018D000330382179307B1F030933303209332031D
:1018E000E0912C05F0912D05309761F00084F18591
:1018F000E02D309739F083E089833B832A83CE0142
:10190000019609952396E2E00C949332A3E0B0E0AF
:10191000ECE8FCE00C9477329C01809130039091CC
:10192000310382179307B1F03093310320933003D2
:10193000E0912C05F0912D05309761F00084F18540
:10194000E02D309739F084E089833B832A83CE01F0
:10195000019609952396E2E00C9493329C01FC01D8
:1019600032968FEF90E04191461751F08F3F19F476
:10197000411101C0892F9F5F9630A9F78F3F09F46D
:101980000895280F311D87FD3A95F9016283089566
:10199000E0E1F3E09191891302C0DF011E9293E030
:1019A000E631F907B9F7089580910B0108952FB733
:1019B000F89480912C0390912D03A0912E03B09167
:1019C0002F032FBF0895F3DF2091590530915A0559
:1019D000232B211521F08093080590930905209170
:1019E0005B0530915C05232B211521F080930605C2
:1019F00090930705E0912C05F0912D05309759F053
:101A00000680F781E02D309731F082E08093570512
:101A100087E595E009950895611509F441C0E3E370
:101A2000E80FE33148F4F0E0E35EFB4C0C94C53280
:101A3000C6DE819580935A05C6CFC1DEFBCFBFDEDF
:101A4000819580935905F8CFBADEFBCFD8DE80931D
:101A50005B05F2CFD4DE8195FACFD1DE81958093FC
:101A60005C05EACFCCDEFBCF815D990B21E030E055
:101A700001C0220F8A95EAF780915805822B809346
:101A80005805DACF80915605816080935605D4CFF2
:101A9000809156058260F9CF809156058460F5CF1C
:101AA000409159058D3C59F480915A0587FF0DC02E
:101AB00010925A05411559F41092550508C08E3CF4
:101AC00081F480915A0518169CF3411581F080919C
:101AD0005B0590915C05892B8111AECF1092540566
:101AE000ABCF8F3C41F447FFF0CF10925905809166
:101AF0005A058115E0CF803D19F41416B4F3E5CFF3
:101B000090915B05893D29F41916FCF610925B054E
:101B1000DCCF8A3D19F497FFD8CFF8CF90915C05C0
:101B20008B3D29F497FFD1CF10925C05CECF8C3D31
:101B300019F41916CCF3C9CF9FE2980F983090F49E
:101B4000815D990B21E030E0B90102C0660F771F7B
:101B50008A95E2F7CB01809590915805892380936F
:101B60005805B3CF8D3D31F4809156058E7F80931B
:101B70005605ABCF8E3D21F4809156058D7FF7CF72
:101B80008F3D09F0A2CF809156058B7FF0CF2FB704
:101B9000F89460912C0370912D0380912E03909105
:101BA0002F032FBF0895CF92DF92EF92FF92CF9332
:101BB000DF93D82FC92FC0904706D0904806E090F9
:101BC0004906F0904A06E3DF6C197D098E099F09EA
:101BD000643F71408105910510F1D9DF6B017C01F3
:101BE00082E390E0A0E0B0E0C0920205D09203054D
:101BF000E0920405F09205058093FE049093FF04A3
:101C0000A0930005B0930105D0934506C093460606
:101C1000DF91CF91FF90EF90DF90CF90089584EF08
:101C200091E0A0E0B0E0E0CF0895FC019B0180913D
:101C30002203909123038617970740F0672B29F41E
:101C40008091E8008E778093E800C90140E000971A
:101C500041F4411106C08091E80082FF2FC080E06E
:101C60000895209123052115A9F12530A9F120918E
:101C7000E80023FD2DC02091E80022FDECCF20914B
:101C8000E80020FFE4CF3091F3002091F2000097AC
:101C900019F02830310558F041E02830310509F0BD
:101CA00040E02091E8002E772093E800D0CF4191CA
:101CB0004093F10001972F5F3F4FE9CF80912305BB
:101CC000811541F0853041F08091E80083FFC3CF5A
:101CD00081E0089582E0089583E0089580911C03D7
:101CE00087FF13C08091E80082FF06C08091E80062
:101CF0008B778093E8000895809123058111F2CFBE
:101D00000895809123058115D9F38091E80080FF23
:101D1000F8CF8091E8008E77ECCF2091E4003091ED
:101D2000E50095E6A9012091EC00822F817020FF4B
:101D300006C08091E80080FF06C080E008952091F1
:101D4000E80022FD1AC080912305811589F08530B5
:101D500089F08091EB0085FD0FC02091E400309167
:101D6000E50042175307F9F29A95E1F684E00895E9
:101D700082E0089583E0089581E00895E8EDF0E0C1
:101D800080818E7F80831092E2001092DA001092A0
:101D9000E100A0EEB0E08C9181608C9380818F7720
:101DA000808319BCA7EDB0E08C918E7F8C938081ED
:101DB0008F7E808310921B030895E0912C05F09193
:101DC0002D05309739F00284F385E02D309711F01E
:101DD00060E209950895EF92FF920F931F93CF93BE
:101DE000DF937C01809104015BDBC82F192F609188
:101DF00013056695669521E0620F08F46FEF8091F8
:101E00004504909146048CD8082FD0E0C11748F0C3
:101E100081E0153508F080E0CDB7DEB7E6E00C9440
:101E20008F32FE01E95BFD4F80819091050189238E
:101E3000811581F060911005709111058091120556
:101E4000202F4C2FF70109950E940107472F282FBB
:101E5000CE0122DB2196DACFA0E0B0E0E2E3FFE0A2
:101E60000C946B323C01809104011ADBC82F192FAE
:101E7000609113056695809145049091460450D871
:101E8000F82ED0E0CE01880F991F9C0123563E4FBB
:101E900069011C1709F048F481E0153508F080E06D
:101EA000CDB7DEB7EEE00C948732FE01E95BFD4F63
:101EB0008081909105018923811561F1F60180816E
:101EC000282F2057330B59018181E82FE052FF0B57
:101ED0004F01AA9C9001AB9C300D300D1124EE9F58
:101EE000C001EF9F900D900D1124820F931F25D8F4
:101EF000082F609110057091110580911205EF2C4B
:101F00009401A501F30109950E940107472F282F8D
:101F1000CE01C2DAF2E0CF0ED11C2196BACFAF9239
:101F2000BF92DF92EF92FF920F931F93CF93DF93B5
:101F30005C0180910401B4DAC82F192F6091130558
:101F4000669580914504909146040E949007D82E92
:101F5000D0E0CE01880F991F9C0123563E4F790196
:101F60001C1709F070F481E0153508F080E0DF916E
:101F7000CF911F910F91FF90EF90DF90BF90AF90A6
:101F80000895FE01E95BFD4F808190910501892351
:101F90008115B1F0F70121812052330B4081405768
:101FA000550B6091100570911105809112050D2D52
:101FB000F50109950E940107472F282FCE016CDA01
:101FC000F2E0EF0EF11C2196CBCFA0E0B0E0EBEEFB
:101FD000FFE00C9470328C018091040161DAC82F0B
:101FE000D92E2091130531E0230F08F42FEF30E0B4
:101FF00040E050E06FEF7FEF80E090E00E94BE3362
:102000007901D0E0C22EBF2C2C2FCD1550F081E0ED
:10201000F5E5DF1608F080E0CDB7DEB7E9E00C9417
:102020008C32FE01E95BFD4F80819091050189238F
:10203000811509F1409154044150042E000C550BB8
:1020400047FF1BC08C2D9B2D6091130521E0620F73
:1020500008F46FEF0E949007AC0160911005709139
:10206000110580911205F80109950E940107472F7B
:10207000282FCE0111DA2196C7CFFA01EC5AFB4F77
:10208000818982130AC0FA01EE0FFF1FEC5AFB4F41
:10209000818D928D8E159F05B8F241505109D0CF98
:1020A000A8E0B0E0E6E5F0E10C946732382E6A83F0
:1020B0007B8380910401F4D9192F209154042E833D
:1020C000E82FF0E0F887EF83CF01880F991F9C017C
:1020D00023563E4F6901432C512C3FEF431A530ABC
:1020E0008F81811740F081E0153508F080E0289657
:1020F000E2E10C948332EF81F885E95BFD4F80814A
:102100009091050189238115E9F0809110058C8358
:10211000909111059D83F201EC5AFB4F3F01232C56
:102120001982FE812F16C0F06091120589810E94EC
:1021300088076C817D810E940107472F282F8F819E
:102140009885AAD92F8138852F5F3F4F38872F83F5
:1021500032E0C30ED11CC4CFF30181913F01F601DF
:10216000A080A81ABB088180F3018781881A99088A
:10217000AA9C9001AB9C300D300D1124889CC001AD
:10218000899C900D900D1124820F931F0E949D0732
:10219000082F6091130521E0620F08F46FEFF3013F
:1021A000EE0FFF1FE455F440858996890E94900741
:1021B0007C019401A5016C817D818981EA81FB818B
:1021C00009956C837D8389832394ABCF982F90935B
:1021D000E900891771F07091EC002091ED005091A9
:1021E000F00021FD09C09F5F973089F78093E900D7
:1021F0000895762F242F50E03091EB003E7F3093EE
:10220000EB003091ED003D7F3093ED003091EB001D
:1022100031603093EB007093EC002093ED0050930D
:10222000F0002091EE0027FDDECF0895A0E0B0E0A1
:10223000ECE1F1E10C947132C8EDD0E088818F7E41
:102240008883E7EDF0E080818160808384E082BF55
:1022500081E080931B0388818E7F888302EE10E0EB
:10226000F80110821092DA0081EEC82ED12CF6010E
:10227000108288818F7788838881806888838881AD
:102280008F7D888319BC1092230510921A03109237
:102290007E041092190390EEE92EF12CF701808153
:1022A0008B7F808388818160888342E060E080E06A
:1022B0008DDFF60180818E7F8083F80180818160CF
:1022C0008083808188608083F70180818E7F808316
:1022D000888180618883CDB7DEB7E8E00C948D32C9
:1022E00031B33E7F21B321604FB7F89484E393E08C
:1022F000FC010196508168E021BB000000C057FF3F
:1023000031BB550F000000C000C000C031BB00C091
:102310006A9591F754E08333950751F74FBF8FE5E6
:1023200094E00197F1F700C00000089581E08093E8
:10233000E00080E28093D8001092C9008FE19EE413
:102340000197F1F700C0000087E090EBDC0180937B
:10235000CE069093CF06A093D006B093D10688E125
:102360009CE00FB6F894A895809360000FBE909300
:102370006000FFCF0F931F93CF93DF938B01EA0190
:1023800090912305943051F58093E9008FEF90915F
:10239000E80095FD06C095ED9A95F1F700008A9545
:1023A000B1F78091E80085FF19C0B7DC811111C039
:1023B0008091E80085FD06C08091E8008E778093CB
:1023C000E800F3CFF80181918F018093F10021970C
:1023D00079F78091E8008E778093E800DF91CF91C4
:1023E0001F910F910895792F603229F440E250E057
:1023F000682F82E0BFCF0895CF93DF93D82FC92FE6
:1024000048E050E0682F792F81E0B4DF88E0ED2FBD
:10241000FC2FA4E2B3E001900D928A95E1F7DF91E1
:10242000CF910895BC0146E050E084E0A3CFBC0109
:1024300043E050E084E09ECF1F93CF93DF93962F2D
:10244000122F632F8430D8F49530C8F44F30B8F48D
:10245000C42FD0E0CC0FDD1F2EE1929FC00DD11D07
:10246000112496E9899FC00DD11D1124CE018996B2
:102470000E948933612FCE018A960E948933DF91B1
:10248000CF911F9108959091CD068091CC06982B05
:102490008091C905809589239091C805892B8093E7
:1024A0000E0348E050E06EE275E08EE093E00E949B
:1024B0004033892BB9F088E0EEE0F3E0AEE2B5E01E
:1024C00001900D928A95E1F7E0912C05F0912D0590
:1024D000309741F00280F381E02D309719F08EE0C3
:1024E00093E009950895CF93C6E0E0E1F3E0DF01C2
:1024F0008C2F1D928A95E9F780E090E0DFD980E08B
:1025000090E004DA1092CC06BEDFE7E5F5E0DF01EB
:102510001D92CA95E9F71092550510925405109234
:10252000560551DACF9108951092CD06DCDF2FEFDA
:1025300084E39CE0215080409040E1F700C000001F
:1025400088E19CE00FB6F894A895809360000FBED8
:1025500090936000FFCFAAE2B0E0E1EBF2E10C94CF
:1025600076328CE193E0FC0101962091F10020830A
:1025700023E084329207B9F780911D03893009F472
:1025800059C0C8F4823009F4B4C0833009F484C05F
:10259000813091F18091E80083FFE8C080911C03B5
:1025A00090911D039A3008F0E1C0E92FF0E0E05D62
:1025B000FB4C0C94C5328A3009F48BC08B3051F738
:1025C00080911C03813231F7809120039091210387
:1025D000892B01F78091E800877F8093E8007EDBFC
:1025E00081E090911E03911101C080E080930C0165
:1025F0001092CD0678DFCECF80911C03813A51F640
:102600008091E800877F8093E8008091200390917B
:102610002103892B59F060E080E090E070E005DB59
:102620008091E8008B778093E800B4CF68E084E283
:1026300093E0F4CF80911C03813209F0ABCF8091FD
:102640002003909121038D7F892B09F0A3CF8091E6
:10265000E800877F8093E8008091E80082FF17C040
:102660009091F3008091F200029731F48091F10093
:10267000813011F0863021F48091F10080930B01BC
:102680008091E8008B778093E80028DB83CF8091EE
:1026900023058111E1CF7ECF80911C03813A09F09F
:1026A00079CF8091200390912103892B09F072CF7B
:1026B0008091E800877F8093E8008091E80080FFA8
:1026C000FCCF80910C018093F1008091E8008E771F
:1026D000DACF80911C03813209F05CCF8091E80051
:1026E000877F8093E800FADA80911F0380930A01C4
:1026F00051CF80911C03813A09F04CCF8091E800C2
:10270000877F8093E8008091E80080FFFCCF809174
:102710000A01D9CF803889F0823841F580912003B1
:102720008F70873018F58093E9008091EB0085FB6E
:10273000882780F91092E90006C080917E04880FF6
:1027400090911903892B9091E800977F9093E8006E
:102750008093F1001092F1008091E8008E7723C001
:10276000811116C080911E03813009F18091E8002B
:1027700083FF0AC08091E800877F8093E800809102
:10278000EB0080628093EB00AA96E3E00C94923217
:10279000823061F780911E03811581F01092E9006B
:1027A0008091E800877F8093E80098DADFCF81E0AE
:1027B000933009F080E080937E04F0CF8091200375
:1027C0008F702FEF280F263088F68093E900209134
:1027D000EB0020FFE3CF933031F48091EB00806277
:1027E0008093EB00DBCF9091EB0090619093EB0036
:1027F00021E030E0A90102C0440F551F8A95E2F79D
:102800004093EA001092EA008091EB008860E8CFE4
:102810008111ACCF10911E031F778091E300807867
:10282000812B8093E3008091E800877F8093E8000C
:1028300055DA8091E80080FFFCCF8091E30080684A
:102840008093E30083E0111101C082E080932305AF
:102850008DCF8058823008F089CF80911E039091EF
:102860001F038C3D53E0950791F583E08A838AE24C
:1028700089834FB7F894DE01139620E03EE051E2E1
:10288000E32FF0E050935700849120FF03C082951E
:102890008F703F5F8F708A30C0F0895C90E08D93BD
:1028A0009D932F5F243161F74FBF8091E800877FB0
:1028B0008093E8006AE270E0CE010196B6D980917B
:1028C000E8008B778093E80051CF805DE7CF292F18
:1028D00033272330310509F44EC078F52130310516
:1028E00009F488C08BE590E0EDE3F2E02230310599
:1028F00009F03CCF2091E800277F2093E800209149
:102900002203309123038217930708F49C0140E0CF
:102910002115310509F073C0411171C08091E800A3
:1029200082FDCDCF80912305811549F2853039F2A2
:102930008091E80083FFF2CFC2CF80912003909175
:1029400021032132310509F446C02232310509F054
:102950000DCF8330910508F009CFFC01EE0FFF1F6A
:10296000E65DFE4F0190F081E02D895D9E4FDC0118
:102970008C9190E010C09C013327823021F12330EC
:10298000310568F4232BB9F4E4EEF2E0E4918E2FE4
:1029900090E0E4EEF2E0009709F4E8CEABCF23300C
:1029A000310509F0E3CEEAEAF2E0E4918E2F90E0FF
:1029B000EAEAF2E0F0CFE4EDF2E0E4918E2F90E06D
:1029C000E4EDF2E0E8CFE8ECF2E0E4918E2F90E065
:1029D000E8ECF2E0E0CF8330910508F0C7CEFC01CF
:1029E000EE0FFF1FE05DFE4F0190F081E02D89E0CA
:1029F00090E080CF82E190E0E8E9F2E07BCF809147
:102A00002305811509F45BCF853009F458CF8091F7
:102A1000E80083FD54CF8091E80082FD7FCF809154
:102A2000E80080FF75CF9091F3008091F2002115AE
:102A3000310519F08830910550F041E0089709F010
:102A400040E08091E8008E778093E80061CF449168
:102A50004093F1003196215031090196E8CF80383A
:102A600009F084CE8091E800877F8093E800809110
:102A70001A038093F10070CE811178CE10911E035D
:102A8000123008F073CE8091E800877F8093E800D1
:102A900010931A0323D91115D9F084E080932305EC
:102AA00042E061EC81E092DB42E261EC84E08EDBAB
:102AB00042E261EC82E08ADB42E260EC83E086DBAA
:102AC00080912305843051F482E080930D014ECE35
:102AD0008091E30087FDE1CF81E0E0CF81E0F5CF99
:102AE000CF93C82F8115A9F08CEF8C0F813A98F401
:102AF000E0E1F3E086E193E02191C21709F43EC0E2
:102B00008E179F07C9F76C2F8EE093E00E94AE0CE2
:102B1000BADCCF91089580E28C0F883068F4C770DA
:102B200021E030E001C0220FCA95EAF78091CD067E
:102B3000822B8093CD06ECCF8BE58C0F833038F45D
:102B40002C2F2452330BC9010E945E0CE2CFE8E522
:102B5000EC0FEB3150F4F0E0EE0FFF1FEA52FD4FA7
:102B6000808191810E94860CD4CF83E38C0F8331C6
:102B700080F661E08C2F0E940C0DCBCF8C2F0E9431
:102B8000C80C81DCC0CFCF93DF93EC01805E91094C
:102B9000089720F06CE276E1209711F46DE176E180
:102BA000CE010E9431048C2F9BDFDF91CF910895DD
:102BB000811561F19CEF980F913A18F40E94C80CAE
:102BC00062CC90E2980F983050F4877091E001C089
:102BD000990F8A95EAF7892F0E94F704F1CF9BE5B8
:102BE000980F933020F480E090E00C945E0C98E510
:102BF000980F9B3120F480E090E00C94860C93E3D6
:102C0000980F933118F460E00C940C0D08951F9305
:102C1000CF93DF93182FEB0163DF209731F4812FDF
:102C2000C7DFDF91CF911F9108958FE99FE0019752
:102C3000F1F700C000002197F0CF811531F090919D
:102C4000CD06892B8093CD061ECC0895811519F0F1
:102C50000E94F70418CC0895811531F09091CC06AC
:102C6000892B8093CC060FCC0895811539F080957F
:102C70009091CC0689238093CC0605CC0895809151
:102C8000C405811521F082E2F0DF1092C405089599
:102C9000CF93DF93EC0149855A856D857E850E942F
:102CA0004A0C9B8190958091CC0689238093CC0619
:102CB000EADB85E0FE0111928A95E9F7DF91CF9179
:102CC0000895CF93DF93EC018C8181FD10C0826069
:102CD0008C838091CC069B81892B8093CC06D3DB9F
:102CE0004F8158856D857E85CE010E944A0C1092D9
:102CF000C6061092C5068C8180FD02C0CE01C8DFD9
:102D0000DF91CF9108951F93CF93DF93182FA09158
:102D10004306B0914406109709F449C01092460644
:102D2000109245061092C9051092C8051696CD91CD
:102D3000DC911797CE019A9581159F4108F4D07EBA
:102D4000D1E0C11101C0D0E01996ED91FC911A9724
:102D5000309731F01B966D917C9180E00995D823D6
:102D6000D11539F08CEF8C0F813A28F58C2F0E9409
:102D7000C80C1115A9F0E0914306F0914406808536
:102D800084FD0EC080914206811551F080819181B1
:102D90009C01215031092F333E4710F40E94D30D7E
:102DA00072DB109244061092430610924206DF91A5
:102DB000CF911F91089567DB8C2FFADEDACF0F9346
:102DC0001F93CF93DF93843030F5653020F54F307B
:102DD00010F5C42FD0E0CC0FDD1F2EE1629FC00D97
:102DE000D11D112436E9839FC00DD11D1124CE01C0
:102DF00089960E946D33082F10E0102F0027CE0116
:102E00008A960E946D339801282BC901DF91CF91DA
:102E10001F910F91089580E090E0F8CF462F672F23
:102E20002091280530912905232B81F4703F39F436
:102E3000403F61F4809126059091270508957530F3
:102E400028F44F3018F4843008F4B9CF80E090E0D3
:102E50000895A0E0B0E0EFE2F7E10C9472327C015B
:102E60000091CB068091CA06082BC3E0D0E010E0A9
:102E7000C8010C2E02C0959587950A94E2F780FD53
:102E800009C02197A8F7D12C8D2DCDB7DEB7E7E08B
:102E90000C948E32DC2EB7018C2FC0DF0E94F2051D
:102EA000019779F3F1CF0F931F93CF93FC018681A4
:102EB0009781009789F4858100811181811581F0C6
:102EC000611571F0C801C5DFC82F682FC8010E94C5
:102ED0006E04B8018C2FA2DFCF911F910F9108953E
:102EE000C8010E94A404C82FF4CF382F292FCB018A
:102EF000A32FB22F8F3A9105A105B10520F48F5A67
:102F00009C4F0C946D3380E0089585E290E00E9420
:102F10006D338D3289F486E290E00E946D338D32FC
:102F200059F487E290E00E946D3391E08C3009F013
:102F300090E0892F8170089580E0FCCFAAE0B0E096
:102F4000E4EAF7E10C946C32C0902105D0902205A0
:102F500081E090E09093220580932105812C912CB3
:102F6000E12C5401F12C14C0F80125913591472D25
:102F70006F2D8E2D61DA0E5F1F4F73948FE07812E4
:102F8000F3CF9FE0A90EB11CF394E5E0FE1639F0F3
:102F90008501000F111F08511D4F712CE5CFE394DF
:102FA000FBE48F0E911C84E0E812DBCF1A821982B9
:102FB0001C821B821E821D8218861F8288EC90E074
:102FC0009A87898701E812E0FE0131967F014AE085
:102FD00050E0B801C7010E94A733065F1F4F013DB3
:102FE000F2E01F07A1F789E0F70111928A95E9F74E
:102FF0008FEF9FEF9E838D8387E08A874AE050E0C2
:10300000B801C7010E94A733065F1F4F0132F3E0EA
:103010001F07A1F786E0F70111928A95E9F746E0CC
:1030200050E0B801C7010E94A7330A5F1F4F013566
:10303000F3E01F07A1F7D0922205C09221052A963E
:10304000EDE00C948832AAE0B0E0E9E2F8E10C94FB
:103050006F320AEC15E081EDE82E82E0F82E97E061
:10306000B92E23E3C22E24E0D22EAA24A3944AE050
:1030700050E0B701CE0101960E945D33F801389609
:10308000DF018B2D1D928A95E9F789819A81D801FC
:1030900011969C938E938F8112968C9312978D81AB
:1030A00013968C931397888514968C93149789851F
:1030B00015968C9315978B819C8117969C938E9374
:1030C00016978A8587FD04C01E96DC92CE921D97C6
:1030D00080FF02C0F801A08681FF07C0D8011896C2
:1030E0009C911897926018969C9382FF04C0F801F7
:1030F00090859460908783FF07C0D80118969C91B3
:103100001897986018969C9384FF04C0F8019085E6
:103110009061908785FF07C0D80118968C91189709
:10312000806218968C93BAE0EB0EF11C015F1F4F82
:10313000E1E2EE16E3E0FE0609F099CF2A96EAE016
:103140000C948B32A6E0B0E0E8EAF8E10C9472321D
:1031500006E615E081E2E82E83E0F82E98E0D92E0D
:1031600046E050E0B701CE0101960E945D33F801C0
:103170008D2D11928A95E9F7B8016C5F7F4F898197
:103180009A810E94360BF80191838083B8016B5FAE
:103190007F4F8B819C810E94360BF8019383828341
:1031A0008D8186838E818783F6E0EF0EF11C085FA8
:1031B0001F4F81E5E81683E0F80691F62696E7E0D2
:1031C0000C948E32282FCB01283070F44AE0249FD3
:1031D00090011124B9016F577D4F4AE050E00E94E1
:1031E0005D3380E090E008958FEF9FEF0895AAE0AF
:1031F000B0E0EDEFF8E10C946B32FE0131968AE01D
:10320000DF011D928A95E9F79EE3A92E91E0B92E80
:103210008F013F01EE24E394F12C32E5C32E31E01F
:10322000D32EF50181915F018F3F09F444C0F894DA
:10323000E82FE295EF70F0E021A18F70A70102C0A6
:10324000440F551F8A95E2F7CA01922F982B91A33C
:1032500092A18095892382A3789400C0E3E4F1E0F1
:1032600021E030E0812C912C41914F3F79F0A42F47
:10327000A295AF70A05EB0E08C9190E04F7002C05C
:10328000959587954A95E2F780FF3BC080E090E0F6
:10329000882A992A220F331FCE16DF0629F7F50157
:1032A00082918F3F11F00E94E80650EA5A95F1F79B
:1032B000D8018D929C920E5F1F4FB3E4AB16B1E024
:1032C000BB0609F0AECF4AE050E0B30189E494E0D8
:1032D0000E944033892BB9F08AE0F301A9E4B4E0FD
:1032E00001900D928A95E1F781E0809318030E9486
:1032F000D70C90931703809316032A96EEE00C9454
:103300008732C901C5CF809118038115B1F30091AF
:103310001603109117030E94D70C801B910B059781
:1033200060F34AE050E069E474E087E195E00E94D0
:103330004033892B49F08AE0E9E4F4E0A7E1B5E005
:1033400001900D928A95E1F710921803D6CF48E0CC
:1033500050E067E170E08FE095E00E947A331092D0
:1033600053040895EFE0F5E085E3808380911B012D
:1033700090911C01A0911D0181839283A3838FE70B
:1033800084838FEF8583E3CFA3E0B0E0EAECF9E13B
:103390000C946732C0903C04D0903D04E0903E0411
:1033A000F0903F040E94C70D2B013C0153014201E4
:1033B0008C189D08AE08BF080E94C70D60933C049E
:1033C00070933D0480933E0490933F04A091CA04FF
:1033D000EAECF4E04A2F50E02FEFC20ED21EE11CBF
:1033E000F11CC418D508E608F708A5132BC04093B4
:1033F000CA0420910F05322F3370432E311519F076
:10340000422E4694469430910901323009F46AC341
:1034100048F531112EC01092040160934504709359
:103420004604809347049093480489E2EAECF4E070
:10343000A4E5B4E001900D928A95E1F781E08093D4
:10344000090113C0218D328DC216D306E104F104A7
:1034500020F441505F5F3296C8CF280D391D328F5E
:10346000218FF8CF333009F445C32396E2E10C9461
:10347000833280910801481221C0237040910701D6
:1034800050E081E02417150609F480E080930601DE
:103490008091140590910501981739F080930501EA
:1034A00040E060E080E00E944E0A41E2441688F469
:1034B000E42DF0E0E65CFB4C0C94C53281E0E6CFF5
:1034C00080910601811529F040E060E080E00E94D3
:1034D0004E0A80E00DC1809104010E94500A898348
:1034E000192F6091100570911105809112050E94AD
:1034F0000107062FF72EE82E9981892F90E09B83F4
:103500008A83BA811B1709F018F481E0153543C08E
:10351000EA81FB81E95BFD4F808190910501892360
:10352000811539F02E2D4F2D602F8A819B810E94AD
:103530004C0AAA81BB811196BB83AA83E2CF8091FA
:1035400004010E94500A8983E92EE0911005EA8364
:1035500000911105109112056E2F702F812F0E947E
:103560000107D62EC72EB82E809113056A81680FE9
:10357000702F812F0E940107162F072FF82E3981F7
:10358000232F30E03B832A835A81E51609F030F47B
:1035900081E095E5E91608F4ABC09BCFEA81FB8199
:1035A000E95BFD4F8081309105013823311561F0D1
:1035B0002F2D402F612F80FD03C02B2D4C2D6D2D05
:1035C0008A819B810E944C0A4A815B814F5F5F4FD9
:1035D0005B834A83D9CF809104010E94500A89837A
:1035E000192FF0901105E09012056091130580E409
:1035F0000E948807082FB981AB2FB0E0BB83AA8354
:10360000FA811F1709F008F480CFEA81FB81E95B9A
:10361000FD4F80819091050189238115C1F0EA81D8
:10362000FB81EE0FFF1FE256FE4F808182958F7067
:1036300060911005809F600D11247F2D8E2D0E94BA
:103640000107472F282F8A819B810E944C0AEA811B
:10365000FB813196FB83EA83D3CF809104010E94E2
:10366000500A8983192FF0901105E090120560919E
:10367000130580E40E948807082F3981232F30E04A
:103680003B832A835A81151709F008F43ECFEA815B
:10369000FB81E95BFD4F80819091050189238115B4
:1036A000E1F0EA81FB81EE0FFF1FE356FE4F208120
:1036B000209F9001112465E0359527956A95E1F7E3
:1036C00060911005620F7F2D8E2D0E940107472FFC
:1036D000282F8A819B810E944C0A4A815B814F5F1F
:1036E0005F4F5B834A83CECF8CEF97E00E94EB0E57
:1036F000909104019F5F909304018111B6CE82E006
:1037000080930901809106018111AFCE4110ADCEA9
:1037100083E095CE87E298E0E9CF8FE598E0E6CFA9
:1037200086E998E00E948F0FE3CF82EB98E0FACF12
:103730008DEC98E00E942C0FDBCF87EE98E0FACF5B
:1037400080E099E0D3CF82E099E0D0CF8BE099E0A0
:10375000CDCF84E199E0CACF8DE299E0EBCF8EE343
:1037600099E0E0CF86E699E0DDCF809104010E94E8
:10377000500A682E992E80910601811561F040E073
:1037800060E080E00E944E0AEFE7F4E08BE4DF01A6
:103790001D928A95E9F78091040181111BC0E09187
:1037A0004104F0914204FB83EA830E94D70C2A81F2
:1037B0003B81821B930B21E08931910508F420E0C5
:1037C00020934004499730F00E94D70C9093420414
:1037D00080934104C12CD12C712C4AEA542E22240E
:1037E00023947601812CF701EE5AFE4F3081398304
:1037F000361508F43FC0391508F03CC0432F50E09F
:103800005B834A83FA01E95BFD4F8081909105015A
:103810008923811571F1C70181589B4F5C01DC013F
:103820001C91012F25E5021B08F400E030901105E2
:10383000252D210F08F42FEF822F880F820F609122
:1038400012058E5F0E948807652D601B732D0E94F4
:103850000107472F282F8A819B810E944C0A809163
:103860004004811531F0322D131B08F410E0D5010E
:103870001C9373948394BFEFEB1AFB0AEFE08E1254
:10388000B2CFFCE3CF16D10421F481E045E59416D4
:1038900082CE2FE0C20ED11C31E1731608F4A1CF05
:1038A000F4CF50901205E52CF12CC701880F991F19
:1038B0008E0D9F1D96958795969587959B838A83F8
:1038C0009A8199838FEF90E0B7010E94B232362E31
:1038D00080910601811571F040E060E080E00E9477
:1038E0004E0AEFE7F4E08BE4DF011D928A95E9F7D9
:1038F00010924404809143048F5F809343048FE7C8
:10390000C82E84E0D82EA12CB12C3701EA81FB818E
:103910006E1A7F0A45018601212C80914404822978
:1039200081114BC00E942933853595400CF045C06C
:10393000D6015C92F401EE5AFE4FE081EF3FD9F0E0
:10394000D8012C91F0E0B981B21708F045C030E001
:103950004A815B81241B350B249FC001259F900D5C
:10396000349F900D1124B3010E949E32262F452DC5
:10397000CF010E944C0A2394015F1F4F5FE0850E28
:10398000911C85E02812C9CF9FEFA91AB90AAFEFA1
:10399000CA1ADA0ABFE0AB16B10409F0BBCF8091B6
:1039A0004304381202C010924304809144048F5F94
:1039B0008D31F8F4809344048CCDF8018081811519
:1039C00009F4B8CF851508F0B5CF909143043912AA
:1039D000B1CF81508083AECF2E9DC0012F9D900D21
:1039E00011246A817B810E949E32462F20E060E094
:1039F000BFCF109244042CEA34E084E09FEF950D91
:103A0000B901EFE7F4E0843021F444AD541201C071
:103A100094AFDB014D91BD01451540F08D01015082
:103A20001109D8019C93DB011E965C923196B4E09B
:103A3000EE38FB0741F781502F5031098111E0CF5B
:103A400048CD86E799E00E94E50F52CE83E899E0E1
:103A5000FACF8091540421E0382F321B08F430E073
:103A6000832F65E979E00E94501042CE65E979E044
:103A700080E0F9CF8091540421E0482F421B08F4E4
:103A800040E0842F6EEA79E0EECF6EEA79E0F0CF85
:103A90008091540421E0582F521B08F450E0852FE8
:103AA00066EE79E0E0CF66EE79E0E2CF80915404F3
:103AB00021E0382F321B08F430E0832F68E17AE0F0
:103AC000D2CF68E17AE0D4CF8091540421E0482F2E
:103AD000421B08F440E0842F60E37AE0C4CF60E347
:103AE0007AE0C6CF409208012370209307010E941C
:103AF00070110ECE80915304811129DCC0904504D1
:103B0000D0904604E0904704F09048040E94C70D0E
:103B10006C197D098E099F09603171058105910538
:103B200008F4A3CC10920901A0CCA0E1B0E0EBE92D
:103B3000FDE10C946932FE01319680E1DF011D92B6
:103B40008A95E9F70BE010E091E5A92E93E0B92EF4
:103B50002FEA422E512C612C712C4F01730162010E
:103B6000B1E14B165104610471041CF080E1C82ED0
:103B7000D12CA601B501C4010E947A33AC0CBD1C46
:103B80000D2C000CEE08FF084C185D086E087F082D
:103B90000150104019F76096E0E10C9485326FEF08
:103BA00085E290E00E9489336FEF86E290E00E9408
:103BB00089336FEF87E290E00E94893360E088E20A
:103BC00090E00E948933BAD9B0DF6DE285E290E0DF
:103BD0000E9489336DE286E290E00E9489336CE0B6
:103BE00087E290E00C948933A0E0B0E0EAEFFDE1D9
:103BF0000C947032EC018881811521F1813009F03B
:103C000048C08981813059F48A81239660E570E04B
:103C1000893311F060E070E00E940716ECCF82302B
:103C200029F48A8123960E947015E5CF833029F408
:103C30008A8123960E94D815DECF843041F02296E7
:103C40008111D9CFCDB7DEB7E9E00C948C328A81EF
:103C5000239620E030E09AE0682F6053770BAB01A9
:103C60006A30710560F02115310551F3EFE9FFE08D
:103C70003197F1F700C0000021503109F4CF929F35
:103C8000B001939F700D11249A01260F371F89915F
:103C9000E3CFE82FF0E0E354FE4FB490282F2695B1
:103CA0002695269530E0F901E355FE4FE4908770A4
:103CB000F12C082E02C0F594E7940A94E2F7E0FA9A
:103CC000EE24FF24E0F8F901E356FE4FC490D12C16
:103CD000082E02C0D594C7940A94E2F7C0FACC2407
:103CE000DD24C0F8F901E357FE4F049110E002C053
:103CF000159507958A95E2F701701127E114F104F3
:103D000019F081EE0E947015C114D10419F086EEED
:103D10000E94701560E070E08B2D0E940716C114A0
:103D2000D10419F086EE0E94D815E114F10419F0BF
:103D300081EE0E94D8150115110529F060E070E0B0
:103D40008CE20E940716219656CFAAE0B0E0EBEA7B
:103D5000FEE10C9467327C01DC0114968C91811594
:103D600009F413C161E0C7019ED88C01F701858178
:103D7000811539F18091C5069091C606009709F129
:103D800008171907F1F09C013327887F9927E0E095
:103D9000F0E0892B41F48FE0829FF001839FF00DCA
:103DA0001124E35BF94F8481846084831183008351
:103DB000CF010E9461161092CC0661E0C70173D852
:103DC0008C018091B90581111BC0D70115968C918A
:103DD000811509F4A0C00034B2E51B0708F087C0C4
:103DE0000115E2E51E0760F40115F7E01F0741F039
:103DF00008F062C0C801805E9109089708F061C0B0
:103E0000D70115968C91811509F439C2C8019757CD
:103E10008038910508F0A6C2003108F0B6C06EEAFD
:103E200070E080E090E061D88111AFC0C12CD12C4E
:103E300076010111A0C134E0332E8E010F5F1F4FB8
:103E4000D801E32D1D92EA95E9F746015701FFEFEE
:103E50008F1A9F0AAF0ABF0AC701B60146D88983E5
:103E6000811509F492C0813009F006C2260137019C
:103E700022E0420E511C611C711CC501B40135D8F1
:103E8000282E8A83811509F480C08FEF820D83303C
:103E900008F085C1C301B20128D88B83811511F0C8
:103EA000C801A2DE4601570133E0830E911CA11C1C
:103EB000B11C75016401C4CF01153FE0130709F47B
:103EC0009FCF2091CD068091CC0698E0F701A7EA1C
:103ED000B5E001900D929A95E1F71093AE0500932D
:103EE000AD051092B005822B8093A60589CF003EC8
:103EF00042E5140750F4003C52E5150708F080CF66
:103F0000C80180569245809779CF980127573C4742
:103F100025303105B0F609379CE71907D1F5209116
:103F2000AD053091AE05232B81F18115A1F081E023
:103F30000E94240C8091A6050E942C1688E0E7EAD6
:103F4000F5E0AEE5B5E001900D928A95E1F780913C
:103F5000B00580935D0586E0F701AEE5B5E0019020
:103F60000D928A95E1F780915D058093B9058EE504
:103F700095E0EBDE1092B905D70115968C91811171
:103F800004C08091A6050E9435162A96E2E10C94A1
:103F900083320A37BCE71B0709F032CF811509F4D9
:103FA000C2C0A090AD05B090AE05E091A605ED832E
:103FB000E983BE016F5F7F4FC5010E94360B2C0164
:103FC000F981F98746E6C42E45E0D42E01E010E0E1
:103FD00022242A94D60117963C90179733FE53C09B
:103FE0006D907C90119712968D909C90139746142B
:103FF0005704B9F41496BC91BF83232DF601468172
:104000006B2F89850E94500B811559F08F810E947A
:104010003A04281634F4D60115969C918401192B84
:10402000282E48145904C9F431FE17C0F601F58151
:10403000FF83232DD60116964C916F2F89850E9400
:10404000500B811551F08F810E943A0428162CF4F0
:10405000F60194818301192B282E30FE14C0FFEF46
:104060002F1211C00130110571F4232DD6011696BF
:104070004C9160E089850E94500B811521F0F6017A
:1040800085818401182BF8E0CF0ED11C26EA35E09B
:104090002C153D0509F09ECF01301105C9F58D8124
:1040A00082958F703D81832B8F7011E0303108F441
:1040B00010E01295107F182BC5019A9581159F412C
:1040C00008F51B29BB240A2D812F8D704A2D8115DF
:1040D00009F44DC06AE082E997E00E94350C282F70
:1040E00030E02115310551F4402F6EE18CE697E068
:1040F0000E94350C282F30E0811541F0C901912B29
:104100008C0106C0A11451E0B506E8F200E010E011
:1041100086E0E1EBF5E0DF011D928A95E9F7109367
:10412000B8050093B7058091B7059091B805892B24
:1041300009F42BCFF7018581811539F08FEF0E94AB
:10414000240C8091B0058093AF0586E0F701A1EBC8
:10415000B5E001900D928A95E1F78091AF058093CB
:10416000B90581EB95E0F1DD1092B9050ECF68E05D
:104170008AE897E0B2CFBFEACB16D104E104F1049C
:1041800009F403CFC701B6010E947517EFEFCE1AED
:10419000DE0AEE0AFE0A8111EECF01504ACE8BEF05
:1041A000820D833090F54601570143E0840E911C47
:1041B000A11CB11CC301B2010E9475178B8381152C
:1041C00009F477CEC501B4010E9475178C83811163
:1041D00008C04601570154E0850E911CA11CB11C7A
:1041E00068CE8B819C818130AFEF9A0710F0982FB9
:1041F0008827B6E02B1629F0E7E02E1621F086D6A8
:10420000E8CF31D6E6CF50D6E4CFF4E053014201F7
:104210002F124FCEC301B2010E947517782E4601AE
:10422000570124E0820E911CA11CB11CC701B601EC
:104230006D5F7F4F8F4F9F4F0E947517711409F468
:10424000A4CE811509F4A1CE8150990B4FEF489F60
:104250009001499F300D1124472D4150550B240FDB
:10426000351F2150310908F424CE8FE99FE00197D2
:10427000F1F700C00000F5CFC801B6DC1ACE011579
:10428000A7E51A0708F487C00115B8E51B0708F071
:104290008FC56801E7E5DE1A6AEB75E08C2D0E9498
:1042A000E218892B19F58FE08C9DF0018D9DF00DA2
:1042B0001124E35BF94F82818130D9F58091BA05F1
:1042C0009091BB05892B91F08091BC059091BD0523
:1042D000892B61F08091BE059091BF052091C005AA
:1042E0003091C105822B932B892B59F18091C40504
:1042F000811193C0D70115965C90511409F40BC13C
:104300000E35BCE71B0709F402C10F35ECE71E07A9
:1043100051F00D35FCE71F0709F0FDC080911A012F
:10432000811509F4F4C010921A0180E00E948316EE
:104330002CCE8230D9F68091BE059091BF05892B95
:10434000A9F22FE02C9DC0012D9D900D1124FC01A0
:10435000EF5AF94F20812E7F2083835B994F0E9473
:104360006116C4CF0337FCE71F07A9F48091C40589
:10437000811519F00E943F1608CE1092CD060E94BA
:10438000D70C88579C4E9093C6058093C50581E055
:104390008093C405FACD023A22E5120771F0023B80
:1043A00032E5130739F0013E110539F0053E1105DC
:1043B00009F09CCF25EE30E002C021EE30E02770FE
:1043C000332781E090E001C0880F2A95EAF7209119
:1043D000C7053091C405311571F0D70115963C9190
:1043E000311521F0282B2093C705CFCD809582234E
:1043F0008093C705CACD322F3823311509F47ACFFF
:10440000982F909592239093C7050E94F704F70187
:104410008581811509F4B9CD6DCFD090CD060E946C
:10442000D70C88579C4E9093C6058093C505D7013D
:1044300015968C91811509F45DCF8D2D8D798111A3
:1044400032C0043BB2E51B0709F454CFB0F5003489
:10445000F2E51F0790F4011522E5120708F04ACF94
:10446000063E110509F446CF1092CC060D32110517
:1044700069F482E08093CC0636C0C801805692452C
:104480008034910508F436CF1092CC060E32110517
:10449000B8F50832110520F50E31110520F5C801D7
:1044A00004974A9730F30E943F168091CD06909171
:1044B000C705892B8093CD061DCF09373CE713072D
:1044C00050F407374CE7140708F014CFC801805C9C
:1044D00092458097D7CF0B375CE71507A9F60ACF2F
:1044E0000A32110501F78091C705811531F08091DD
:1044F000CC0692E089278093CC060E944312FACE24
:104500000C34110581F30D3282E01807EBCF81E006
:1045100080931A013ACD80911A01811143C0C801DC
:1045200097558115914008F0D1C05801F8EFAF229E
:10453000BB24A114B10409F028CD2FE0029FF001A3
:104540001124AF01435B594F6A01D70115968C9135
:10455000EF5AF94F908180FB90F99083811509F40F
:10456000B5C10E94D70C9093C8068093C706F60188
:1045700082818F5F82838091CC069091CD06892BBA
:1045800083834581568165857685C6010E944A0CE4
:10459000D60114968C9181FF5801B092C606A09264
:1045A000C50694C0380130EE631A71083090CD060C
:1045B00048E06416710408F05CC098012770332746
:1045C00081E090E001C0880F2A95EAF7511409F4C0
:1045D0004DC0382AD7018D919C910E94A40421E0FE
:1045E00030E0F90102C0EE0FFF1F8A95E2F7F8876D
:1045F000EF8320914306309144063E832D83409102
:104600004B0650914C065A8749879AECC92E95E083
:10461000D92EA12CB12C311005C0D60112968C9147
:10462000811119C0F601838190E02F8138858223A2
:104630009323892B81F08085982F9770911101C069
:1046400087E038E06316710408F006C1511409F4DC
:1046500063C081FD63C09FEFA91AB90AAFE0CA0E1B
:10466000D11CB8E0AB16B104B1F61CC0809538225D
:10467000B1CF51103EC080914B0690914C06081767
:10468000190781F410924C0610924B0610924706BF
:10469000109248061092490610924A061092460659
:1046A000109245068091430690914406009709F4C4
:1046B00036CFE8E06E16710408F0F2C0632D0E9458
:1046C000960B811103C081E00E948316F70195814A
:1046D0008091CD068272F801911509F430C1E05243
:1046E000F847EB30F10508F055C1E55AFB4C0C9446
:1046F000C53210934C0600934B060E94C70D609381
:104700004706709348068093490690934A06109294
:104710004606109245065ECF82FF9DCFD6018D9052
:104720009C900815190519F4511409F494CFED81E2
:10473000FE81EC15FD0509F48ECFD6011D96ED9195
:10474000FC91309721F08081811509F484CF632D8D
:10475000C6010E94960B811509F47DCF81E00815F2
:10476000190509F080E0482E45208114910441F09C
:10477000411006C0E985FA858E169F0609F06BCFB9
:1047800080E00E948316D0924406C092430681E0E6
:10479000809342068FE08A9DF0018B9DF00D1124DD
:1047A000E653FA4F85818093C90541100EC08114EC
:1047B000910459F0808191819C0124503109213A62
:1047C000310508F04FC00E94C80C8FE08A9DF001AF
:1047D0008B9DF00D1124E653FA4FC680D780C60199
:1047E0009A9581159F4110F420EED222992493943A
:1047F000C60101978F339E4708F0912C8FE08A9D68
:10480000D0018B9DB00D1124A653BA4F1996ED918E
:10481000FC911A97309731F01B966D917C9181E055
:10482000099598229114A9F08FE08A9DF0018B9D43
:10483000F00D1124E653FA4F868197810E940704F8
:104840008093C805C60148E06416710470F40E94A4
:10485000D30D0E94431212C0511409F4FCCE80FD06
:104860005DCFF9CE0E94D815B0CF0497813A91055B
:1048700058F46C2D8EE093E00E94AE0C411409F4C4
:104880004ECE0E94431281CB0E9443128FE39CE9DB
:104890000197F1F700C000008C2D0E947015EECF3B
:1048A000DC012D913C910217130741F4511009C00E
:1048B0001092420680E00E94831631CE511409F412
:1048C0002ECEFC01808585FD2ACEF4CFFA014385EA
:1048D000548565857685C6010E944A0CD6011496DA
:1048E0008C9181FFF3CEC6010E9448168091C506C7
:1048F0009091C6060817190709F0E8CE1092C6066F
:104900001092C506E3CE0E94590A3FCB811559F19A
:104910000E94A30A3ACB811559F10E94C40A35CBF3
:10492000811559F10E94D90A30CB811559F10E94A5
:10493000F10A2BCB811559F10E94070B26CBE054CD
:10494000F847ED30F10530F5EA59FB4C0C94C532CF
:104950000E94630A81E00E94460A17CB0E94710AF6
:10496000F9CF8115A9F20E94990A0FCB8115A9F2FE
:104970000E94BB0A0ACB8115A9F20E94CD0A05CB81
:104980008115A9F20E94E50A00CB8115A9F20E94C7
:10499000FD0AFBCA0737FCE71F07F9F008372CE7C9
:1049A000120749F19801205E32452032310528F581
:1049B000911123C00F7181E090E0AC0102C0440F5F
:1049C000551F0A95E2F78A01642F83E090E00E9468
:1049D0008933802F0E945004D8CA81E0911519F0C4
:1049E0000E94560402C00E94600443E062E081E03D
:1049F0000E94D804CACA82E0F1CF8091C906D09043
:104A0000CB062D2D30E02095309550E0282335231E
:104A1000232B19F08D218093C9060B375CE715070E
:104A200049F4911509F4B1CA8D2D0E943D040E94EC
:104A3000B70BABCA003482E5180750F50032A2E587
:104A40001A0760F59801305521153240E0F19115B3
:104A500009F45EC00130ECE71E0709F457C00330CB
:104A6000FCE71F0709F44CC001152CE7120709F0F9
:104A70004FC01092CD060E9473123FEF44E35CE0FA
:104A8000315040405040E1F700C000000E949611B4
:104A90009801205C324520323105C8F6802F8F7195
:104AA0002091C90630E041E050E0082E02C0440FDA
:104AB000551F0A94E2F724233523232B41F2911545
:104AC00009F463CAB4CF980185E0369527958A9595
:104AD000E1F7822F8F702091C90630E041E050E06D
:104AE000082E02C0440F551F0A94E2F724233523F1
:104AF000232B09F4ACCF91119ACF1092CD06C1CEE1
:104B00006FEF7FEF80E090E00E94A3330E94941249
:104B1000D70116962D913C9121153105C9F0C90197
:104B20000E94F205182FD70115966C91892F829556
:104B30008F70883009F490C040F5843009F471C05A
:104B4000F0F48230A0F160E0C7010E9453171DCA43
:104B5000F701A080B180911569F0C5010E94291765
:104B6000182F682FC5010E946E04B501812F0E9485
:104B70000E17D6CFC5010E94A404182FF6CF85309A
:104B800011F7812F0E940C0DDECF893009F4D5C0BA
:104B90008A5F8F708230B8F6123F09F0E0C0892F2B
:104BA0008F71611509F4E4C00E946004CCCF092F15
:104BB0000F70903110F00295007F6115C9F001155A
:104BC00069F080E2810F883010F011110BC08091E4
:104BD000CD06802B8093CD060E944312812F0E9428
:104BE0007015B1CF8091CC06802B8093CC06F4CF8A
:104BF000812F0E94D815011509F4A5CF80E2810FFD
:104C0000883010F0111106C0802F0E94F7040E9416
:104C1000431299CF00958091CC0680238093CC06D7
:104C2000F6CF892F869586958370811561F0813046
:104C300009F089CF812F9370611102C080E090E06C
:104C40000E94860C80CF812F9370611102C080E09A
:104C500090E00E945E0C77CF892F8370811136C05F
:104C6000611129C0812F829586958770880F880FE2
:104C7000212F2F70082E01C0220F0A94EAF7412F2E
:104C8000407114FF07C04FE050E001C0440F8A9507
:104C9000EAF74095969596959370923091F0842F0F
:104CA000822B933031F08091CA06913039F0242B59
:104CB00082230E9450040E944F0C45CF822B842BEC
:104CC000F8CF242B8091CA068227F3CF611589F192
:104CD00090FFF1CF812F829586958770880F880F7E
:104CE000212F2F70082E01C0220F0A94EAF7412FBE
:104CF000407114FF07C04FE050E001C0440F8A9597
:104D0000EAF74095969596959370842F822B8D2582
:104D1000923061F0842F822B933041F0842F822BCC
:104D20008D21913019F48D2D822B842B0E945304F8
:104D3000C2CF823008F4BFCFCDCF092F0F706115DD
:104D400039F0802F0E945604812F0E941D16B3CF88
:104D5000812F0E942616802F0E946004ACCF133F43
:104D600051F0113FA1F4892F8F71611509F41CCF07
:104D70000E945604E8CE80E0611531F09F7181E019
:104D800001C0880F9A95EAF70E945304DCCE6111A6
:104D900025CF193349F4BFEFE7EEF3E0B150E0401F
:104DA000F040E1F700C00000812F0E94D815CBCE63
:104DB00003372CE7120709F4E8C898CAAEE0B0E060
:104DC000E4EEF6E20C94723249875A876B877C874F
:104DD0008D879E8791111092CC0618861F8286E0DF
:104DE000FE0139968E010F5F1F4FD80101900D9281
:104DF0008A95E1F7FD84D02EE12EF11449F0FD8271
:104E000061E0C8010E94531761E0C8010E94531776
:104E1000FD828D2D9E2D0E94A51E2E96E7E00C94FE
:104E20008E32A6E0B0E0E7E1F7E20C9475320E9422
:104E3000D70C8C0180912A0590912B058017910742
:104E400071F019821A820E94D70CBC0149815A81E3
:104E500080E090E0B3DF10932B0500932A0526969F
:104E6000E4E00C949132A6E0B0E0E9E3F7E20C94C0
:104E700077329093270580932605811520E29207CB
:104E800030F40E94C3152696E2E00C94933280EF32
:104E900089838A830E94D70C8160BC0149815A8131
:104EA00081E091E08BDFEFCFA6E0B0E0EAE5F7E24A
:104EB0000C9475328C01909327058093260501157B
:104EC00080E21807B0F4802F0E94D815C801805ED8
:104ED0009109089728F065E376E10115110511F4B1
:104EE00066E276E1C8010E9431042696E4E00C9463
:104EF000913280EF89838A830E94D70C8160BC0144
:104F000049815A8181E090E059DFEFCFCF93DF9361
:104F1000D82FC92FA8DF8D2F9C2FC6DFDF91CF910F
:104F200008950F931F93CF93DF938C01862F6AEB25
:104F300075E00E94E218892B91F4C091BA05D091D6
:104F4000BB05209761F0F8018281833039F4CE01EE
:104F5000DDDFCE01DBDFCE01D9DF01C0E0F7DF917D
:104F6000CF911F910F9108950F931F93CF93DF93CC
:104F70008C01EB016AEB75E08C2F0E94E218892B03
:104F800009F057C0FE01FF27D80112968C911297A5
:104F9000EC5CFB4F8130A9F414968C9182FD4EC0DD
:104FA00080FF4CC082E080838091BC059091BD055C
:104FB0000097B9F48091BA059091BB050097C9F1AB
:104FC00010C08230A1F514968C9182FD26C080FD20
:104FD0000AC083E080838091BE059091BF05009751
:104FE000F1F041DF26C084E080838091C00590917C
:104FF000C1050097B1F78091BA059091BB05009764
:1050000001F184DF8091BC059091BD05009749F7BF
:105010008091BA059091BB05E4CF85E080838091B3
:10502000BA059091BB05009721F070DFF1CF86E0C3
:105030008083DF91CF911F910F91089581E080834C
:10504000B9CF8091BC059091BD05B8CF0F931F9348
:10505000CF93DF938C01EB016AEB75E08C2F0E94FC
:10506000E218892B71F4DD27CC5CDB4F8881F801D5
:10507000128218828330E9F048F4813059F082308E
:1050800081F0DF91CF911F910F9108958430B1F09D
:105090008530B9F78091BA059091BB05009789F3E7
:1050A00006C08091BC059091BD05009799F3FCDE88
:1050B000E8CF8091BE059091BF05F7CF8091C005E4
:1050C0009091C105009799F72091BA053091BB05E1
:1050D0008091BC059091BD0521153105F9F200972D
:1050E00031F7C901E4CFCDB7DEB7E9970FB6F89431
:1050F000DEBF0FBECDBF85B7806885BF85B780682E
:1051000085BF84B7877F84BF0FB6F894A895809138
:105110006000886180936000109260000FBE80E89C
:1051200090E00FB6F89480936100909361000FBEF9
:1051300081E080930D0186EE96E090930D038093BD
:105140000C030E941E0B0E9423180E94A2180E94AA
:10515000BE0E0E9416118091E20084608093E200EE
:10516000789480912305811599F08091E900109140
:10517000EC008F70179511271795182B1092E900E6
:105180008091E80083FD0E94AB121F701093E9002C
:1051900082E084BD93E095BD9AEF97BD80936E0049
:1051A0000E948517811102C00E94CF1D0EE311E0FD
:1051B000D8018D918D018F3F11F00E94E806B1E07A
:1051C00003341B07A9F703E411E052E5E52E51E093
:1051D000F52EF80181918F018F3F11F00E94E806B2
:1051E000E016F106B1F78AE0E7E1F5E0DF01282FEC
:1051F0001D922A95E9F7E9E4F4E0DF011D928A9512
:10520000E9F780E090E00E947533833E9E4F21F4E1
:105210000E94851781112DC063EE7EEF80E090E043
:105220000E94A33360E082E090E00E94893381E035
:105230008093CA0661E083E090E00E94893360E0D9
:1052400074E184E090E00E94A3330E94B2190E94AE
:10525000CF1D40E050E0BA018FE090E00E949B3308
:1052600040E050E0BA0183E190E00E949B330E944D
:10527000A71982E090E00E946D338093F30484E0EC
:1052800090E00E94753390932505809324050E9439
:10529000F718EFEFF6E721E0E150F0402040E1F7AA
:1052A00000C000000E94F7188091170580FF08C019
:1052B0006FEF7FEF80E090E00E94A3330E94961191
:1052C00083E090E00E946D330E9450040E94710BB5
:1052D0001092540440E150E06FEF70E08DE694E0EE
:1052E0000E9456331092CA0440E150E06FEF70E024
:1052F00083EE94E00E94563381E08093530448E0AB
:1053000050E067E170E08FE095E00E945D3310921D
:10531000530480910F05843010F40E94B2198EE07E
:1053200091E090932D0580932C058091230510E446
:1053300002E1853009F459C10E94F718A4EFB4E0E6
:10534000BAABA9ABE7E1F5E0FCA7EBA74EEF54E061
:10535000DF01E4EFF4E0219131918D919D914E17A1
:105360005F0709F44EC128173907A9F327E135E093
:1053700038AB2FA7C12CD12CF12CAFA5B8A94D90DB
:105380005D90B8ABAFA7E9A9FAA981919191FAAB69
:10539000E9AB8415950509F4E8C09C012425352561
:1053A0003DAB2CABDEA6CDA6E12C66246394712C1C
:1053B0008CA99DA986219721892B09F4C6C0420199
:1053C00086209720E982FA820E94D70C9C838B83E7
:1053D00031E03D8391E08114910409F490E09E83D3
:1053E00049815A816B817C818D81E8DC8114910433
:1053F00041F0EDA5FEA5EE5AFE4F80818F3F09F0EA
:1054000091C2312C032D10E08091CA04830D99279D
:10541000991F09976CF198E0A92EB12CA01AB10A36
:10542000B80165537B4FA5018BEC94E00E944D338E
:10543000B8016D527B4FA50183ED94E00E944D337E
:10544000A501440F551FB801660F771F6D517B4FA3
:1054500083EE94E00E944D33B80165527B4FA50165
:105460008BED94E00E944D3388E083198093CA0449
:10547000311421F14091CA045BA9852F90E0242FBB
:1054800030E0F901E653FB4FDC01AA0FBB1FA35626
:10549000BE4F5C915183880F991FDC01A256BE4F0D
:1054A0008C9181878BA9818BF901EE0FFF1FE65349
:1054B000FB4F128E118E4F5F4093CA04892809F466
:1054C00044C080910F058C7F8C3409F03EC0EDA55F
:1054D000FEA5EE5AFE4F80818F3FB9F1A12CB12C71
:1054E000812C90E09C01220F331FD901A356BE4F9F
:1054F000BFABAEABF901E256FE4FF9AFE8AF2DA559
:105500003EA521583B4F19018501912CF801EE5A17
:10551000FE4F80818F3F59F0F81008C2E91006C293
:10552000D1012C9130E2230F08F42FEF2C939394A8
:105530000F5F1F4FBFE09B12E9CF8394EFE0AE0EE9
:10554000B11CFBE4AF16B104F9F6E394660C771CCA
:105550002DA53EA52F5F3F4F3EA72DA73FE0E312AD
:1055600027CFE9A9FAA952924292F3944FE0C40ED0
:10557000D11C55E0F51201CF0E94C70D47C08091A4
:105580002305843029F10E94C41910927D0448E15A
:1055900050E00FB6F894A895409360000FBE1093AA
:1055A000600083B7817F846083BF83B7816083BFDE
:1055B0007894889583B78E7F83BF0FB6F894A895AB
:1055C00080916000886180936000109260000FBE3F
:1055D0000E94F718E7E1F5E081919191892B09F09C
:1055E000DAC555E0E132F507B9F78091230585303A
:1055F00009F4C5CF1092CD060E9473120E944F0C81
:105600009BCE2817390709F088C10BDC00914506AD
:10561000109146060115110591F1C0900205D09038
:105620000305E0900405F09005050E94C70D6C1974
:105630007D098E099F09C090FE04D090FF04E09080
:105640000005F09001056C157D058E059F05B8F0ED
:10565000C8010E94C315109246061092450610928A
:105660000205109203051092040510920505109290
:10567000FE041092FF0410920005109201050091A3
:10568000C5061091C6060115110509F1E090C7067F
:10569000F090C8060E94D70C8E199F09893C91058D
:1056A000B0F098013327087F112780E090E0012BAC
:1056B00041F44FE0429FC001439F900D1124835B52
:1056C000994FDC0114962C9122FF0E946116809163
:1056D000C405811569F00E94D70C2091C505309151
:1056E000C605821B930B8F3F9F4710F40E943F1605
:1056F0000E94C41986E0E7E5F5E0DE01119601900D
:105700000D928A95E1F7B0905805F0905905D09028
:105710005A05C0905B05E0905C0510925905109207
:105720005A0510925B0510925C058F2D8D2981150D
:1057300009F441C000910805109109050E94D70C99
:105740009C01201B310B90915505911509F41EC544
:105750002531310580F19F3F19F09F5F90935505EA
:10576000F11459F00E94DF0B91E01F140CF09FEF31
:10577000899F802D112480935905D11459F00E94DE
:10578000DF0B91E01D140CF09FEF899F802D1124F9
:1057900080935A0580915905811569F010915A0539
:1057A000111549F00E94D10B80935905812F0E9459
:1057B000D10B80935A058E2D8C29811509F441C097
:1057C00000910605109107050E94D70C9C01201B33
:1057D000310B90915405911509F4D3C4213531054D
:1057E00080F19F3F19F09F5F90935405C11459F0C9
:1057F0000E94FF0B91E01C140CF09FEF899F802DFD
:10580000112480935B05E11459F00E94FF0B91E095
:105810001E140CF09FEF899F802D112480935C054E
:1058200080915B05811569F010915C05111549F0B7
:105830000E94D10B80935B05812F0E94D10B809336
:105840005C05809158058B1119C08091590581150F
:1058500011F0F81213C020915A05211511F02D11E5
:105860000DC090915C05911511F0E91207C03091BF
:105870005B05311103C0822B892B81110E94E30C3F
:1058800086E0FE013196A7E5B5E001900D928A957C
:10589000E1F70E944F0C90910A05891721F080933F
:1058A0000A050E94C70D80912305843009F03DCD83
:1058B00083E08093E9008091E80082FF36CD8091FB
:1058C000E80090E085FF06C00E948D0E811509F466
:1058D00068C091E08091E8008B778093E800911593
:1058E00009F423CD0091280510912905E9810115BE
:1058F000110509F472C0EE3F09F092C08A8183302D
:1059000020F08550833008F08BC0EA81EE3008F03B
:1059100087C0F0E0ED58FB4C38C647E155E058AB86
:105920004FA728CD8BAB332433946CCD90E0EEA9F8
:10593000FFA94081FC01EE0FFF1FE356FE4F2081BF
:10594000421B550BA8ADB9AD2C91880F991FFC01D6
:10595000E256FE4F8081281B330B449FB001459FC8
:10596000700D700D1124229FC001239F900D900D8A
:105970001124860F971F0E949D07382F893208F047
:10598000D6CD28E2231B08F420E0F801E158FB4FB4
:10599000213108F020E13081320F08F43FEF3083ED
:1059A000C6CD00E210E0FE0131967F018091E80053
:1059B00085FD0AC08091E8008B778093E8000E9403
:1059C0008D0E811599F385CF8091F100D7018D93CC
:1059D0007D010150104051F77CCFE43148F4E115CE
:1059E00051F0E150E33138F4F0E0EF57FB4CCDC516
:1059F000EE3F09F48ACF8FEF898312C01A8289E0C3
:105A00008B830EC08A81823081F08330B1F0813087
:105A100091F70E94C70DCFD56B837C838D839E83C6
:105A2000CE0101960E94DD0E80CC88E290E055D632
:105A30001B821C821D828E83F3CF80912105909161
:105A40002205892B69F3FE013196ABA5BCA58C918B
:105A500011969C9111971296BCA7ABA79283838352
:105A60003296A152B54089F7DBCF8A81823009F0A6
:105A7000C2CF6B817C818D819E819DD588E290E033
:105A800048D6CECF4C816B818A810E94DF16982741
:105A9000892798279E838D83C3CF2D813E8132270E
:105AA000232732274C816B818A810E941C12B8CF38
:105AB0000E949E17B5CF8A81823831F178F4803800
:105AC000B1F0813809F0ACCF60E08B810E947D0A93
:105AD0008B81811116C00E94710AA2CF833809F010
:105AE0009FCF8B8120E0409112056C8106C0809190
:105AF000100520E04B816091110590E00E94AC0AF6
:105B00008FCF0E94630A8CCFEB818FE7E43020F4C3
:105B1000F0E0E456FD4F80818093130580E00E9401
:105B2000460A7ECF8A818238C1F050F4803891F0E5
:105B3000813809F075CF80910F058695869560CFE5
:105B4000833809F06DCF809110058B83809111050A
:105B50008C8366CF8091120553CF809113058732D5
:105B600030F08F3530F08E3930F482E049CF80E06C
:105B700047CF81E045CF83E043CF0E94A71950CFA4
:105B800080E18A834DCF1A828FEA3ACF8C818D31A2
:105B900008F046CF8A809B80982489249824A12CE1
:105BA000B12C8E010F5F1F4F7801E80EF11C0E150E
:105BB0001F0509F435CF80E03FEA83169104A10464
:105BC000B10420F4C4018F5A9C4F87D5D801149694
:105BD0008C930F5F1F4FBFEF8B1A9B0AAB0ABB0A58
:105BE000E6CF8091210590912205892B09F418CFE9
:105BF0008C818D3108F014CF882E912CA12CB12CE2
:105C0000CA80DB80DC24CD24DC24E12CF12C8E0145
:105C10000F5F1F4F412C512C3201481459046A0464
:105C20007B0408F0FDCEEFEACE16D104E104F104C6
:105C300038F4D80114966C91C6018F5A9C4F69D5DF
:105C4000BFEF4B1A5B0A6B0A7B0AEFEFCE1ADE0A34
:105C5000EE0AFE0A0F5F1F4FE0CF0E94951DE0CEB7
:105C600084E08FCF8C818D3108F0DACE882E912C94
:105C7000A12CB12CCA80DB80DC24CD24DC24E12CD7
:105C8000F12C412C512C32018E010B5F1F4F481417
:105C900059046A047B0408F0C3CE80E0F8E5CF160F
:105CA000F2E0DF06E104F10418F4C601899615D587
:105CB000D8018D938D01BFEF4B1A5B0A6B0A7B0AEB
:105CC000EFEFCE1ADE0AEE0AFE0AE1CF2C81022F98
:105CD00010E02D3108F0A4CE8A819B819827892776
:105CE00098272C01612C712C8835F2E09F0708F071
:105CF00097CE822E912CA12CB12C48E552E060E089
:105D000070E0441955096609770942175105610584
:105D1000710508F485CE2091210530912205232BB1
:105D200009F03EC01C0129E2220E311C80FBEE244A
:105D3000FF24E0F880FF0BC08896CFD49D8189278F
:105D40009827892781159C4711F48FEF8D83D50102
:105D5000C401840D951DA61DB71D80FF19C06801E3
:105D600041E0C41AD108CE0105968C0D9D1D9CA75B
:105D70008BA7C101800F911FB0D4ABA5BCA59C918E
:105D800081159C4721F48FEFEBA5FCA5808386014C
:105D9000FE013196EE0DFF1D2FEFE016F10638F0F3
:105DA0008E010F5F1F4FC12CD12C760125C094812D
:105DB000858181159C4711F42483258342E0E40EFC
:105DC000F11C3296EACF58E5451652E055066104BB
:105DD000710430F4D80114966C91C201899699D45B
:105DE000BFEFCB1ADB0AEB0AFB0AEFEF4E1A5E0A93
:105DF0006E0A7E0A0F5F1F4FC814D904EA04FB0421
:105E000010F30ECE8091210590912205892B09F483
:105E100007CECE0101960E94DD0EFFEF21EE34E0A9
:105E2000F15020403040E1F700C0000047CA88E050
:105E3000EEE1F1E0DE01919601900D928A95E1F795
:105E4000FE0132968FE1DF011D928A95E9F786E027
:105E5000898388E07F96DE01159601900D928A95E0
:105E6000E1F7DECD8CE2898381E08A831B821C828C
:105E7000D7CD8B819C81092E000CAA0BBB0B25E092
:105E8000880F991FAA1FBB1F2A95D1F7AC01BD012E
:105E9000405E5F4F6F4F7F4F481759076A077B0778
:105EA00008F4BECD8C32E1E09E07A105B10508F0F3
:105EB000B7CD4D32F1E05F076105710520F04CE28E
:105EC00051E060E070E0481B590BBC01605C794F09
:105ED000CE010196CCD3A4CD4AE150E06FEF70E043
:105EE000CE010796E3D38091210589830A831B8223
:105EF0001C8281E08D839FCD81E090E09093290505
:105F00008093280582E390E090930E0580930D0521
:105F10000E94D70C90930C0580930B0581CD011541
:105F2000110581F1D0901705C0901905E0900B057F
:105F3000F0900C050E94D70C8E199F0985369105AB
:105F400040F1C1FE26C0D0FE24C00E94D70C909321
:105F50000C0580930B0580910D0590910E0501971E
:105F600090930E0580930D05892B61F410922905FD
:105F70001092280581E090E09093220580932105FE
:105F800000E010E08091210589830A8380910D054E
:105F900037CD82E390E090930E0580930D05F2CF0C
:105FA00010922205109221053BCD40E250E06FEFA8
:105FB00070E0CE0101967AD333CDEB81E93008F061
:105FC0002FCDF0E0EC56FB4CE0C2FE0132968EE1A4
:105FD000DF011D928A95E9F788E089838B838C83A2
:105FE00083E088A31DCD8C819AE0F92E8E010F5D90
:105FF0001F4FF8012F2D11922A95E9F7B8010E9441
:10600000E2188983F801DE01129601900D92FA944C
:10601000E1F706CD1C818AE0FE013596DE019196FE
:1060200001900D928A95E1F789A19AA10E94110B26
:106030009AA389A38BA19CA10E94110B9CA38BA363
:106040008DA19EA10E94110B9EA38DA38FA198A547
:106050000E94110B98A78FA38FEF183060F43AE0DD
:10606000139FB00111246F577D4F4AE050E0CE01DD
:1060700081966DD380E089830E941E0BD1CC2C8148
:106080006AE0CE018196DC01E62F1D92EA95E9F7E0
:10609000283080F4629FB00111246F527D4F4AE096
:1060A00050E00BD380E089838AE0FE01B196DE01E7
:1060B0001296D3CE8FEFF7CF1C818AE0FE01359682
:1060C000DE01919601900D928A95E1F78BA19CA13A
:1060D0000E94110B9CA38BA38FEF183060F4FAE0A1
:1060E0001F9FB00111246F527D4F4AE050E0CE0156
:1060F00081962DD380E089830E94231891CC2C8136
:1061000066E0CE018196DC01E62F1D92EA95E9F763
:10611000283060F4629FB00111246F5D7C4F46E02F
:1061200050E0CBD280E0898386E0BFCF8FEFFBCFFA
:106130001C8186E0FE013596DE01919601900D925C
:106140008A95E1F789A19AA10E94110B9AA389A3CC
:106150008BA19CA10E94110B9CA38BA38FEF1830E5
:1061600060F4F6E01F9FB00111246F5D7C4F46E0A4
:1061700050E0CE018196EBD280E089830E94A21884
:106180004FCC2B30310508F02ECB5BCB2B303105BB
:1061900008F0E3CA10CB80917E04811509F425CA6A
:1061A00080E189BD09BD09B400FEFDCF8091D80012
:1061B0008F7D8093D8008091E00082608093E00022
:1061C0008091E00081FDFCCF1092CD060E947312F9
:1061D0000CCA1F921FB61F9211248F939F93AF93E7
:1061E000BF9380917D04811113C080912C03909105
:1061F0002D03A0912E03B0912F034196A11DB11D37
:1062000080932C0390932D03A0932E03B0932F0320
:10621000BF91AF919F918F911F901FBE1F901895B6
:1062200078941F921FB61F9211248F939F93AF9360
:10623000BF9380912C0390912D03A0912E03B091D8
:106240002F030196A11DB11D80932C0390932D0364
:10625000A0932E03B0932F03BF91AF919F918F9185
:106260001F901FBE1F9018951F920F920FB60F928E
:1062700011242F933F934F935F936F937F938F934B
:106280009F93AF93BF93EF93FF938091E10082FFC1
:1062900009C08091E20082FF05C08091E1008B7F00
:1062A0008093E1008091DA0080FF24C08091D800C3
:1062B00080FF20C08091DA008E7F8093DA00809189
:1062C000D90080FFA9C080E189BD82E189BD09B400
:1062D00000FEFDCF81E08093230580911B03811197
:1062E00009C00E94BE0E0E9416118091E2008460D7
:1062F0008093E2008091E10080FF1AC08091E2006B
:1063000080FF16C08091E2008E7F8093E200809132
:10631000E20080618093E2008091D80080628093E7
:10632000D80019BC85E08093230583E080930D019C
:106330008091E10084FF2FC08091E20084FF2BC098
:1063400080E189BD82E189BD09B400FEFDCF809165
:10635000D8008F7D8093D8008091E1008F7E80935C
:10636000E1008091E2008F7E8093E2008091E20064
:1063700081608093E20080911A03811509F452C074
:1063800084E08093230580912305843009F052C076
:1063900082E080930D018091E10083FF2CC0809109
:1063A000E20083FF28C08091E100877F8093E100B5
:1063B00082E08093230510921A038091E1008E7F82
:1063C0008093E1008091E2008E7F8093E2008091D3
:1063D000E20080618093E20042E060E080E00E94A1
:1063E000E6108091F00088608093F00081E0809357
:1063F0000D0180930C01FF91EF91BF91AF919F919F
:106400008F917F916F915F914F913F912F910F905D
:106410000FBE0F901F90189519BC10922305109273
:106420001B0368CF8091E30087FF02C083E0A9CF00
:1064300081E0A7CF81E0ADCF1F920F920FB60F92F0
:106440001124EF92FF920F931F932F933F934F933B
:106450005F936F937F938F939F93AF93BF93CF93EC
:10646000EF93FF9309EE10E0F8018081C091EC00FA
:106470008F70C795CC27C795C82B108280EFE82E68
:10648000F12CF7018081877F808378940E94AB1282
:10649000F8011082F701808188608083CF70F80155
:1064A000C083FF91EF91CF91BF91AF919F918F9159
:1064B0007F916F915F914F913F912F911F910F911C
:1064C000FF90EF900F900FBE0F901F9018952F9296
:1064D0003F924F925F926F927F928F929F92AF9274
:1064E000BF92CF92DF92EF92FF920F931F93CF93C1
:1064F000DF93CDB7DEB7CA1BDB0B0FB6F894DEBF58
:106500000FBECDBF09942A88398848885F846E847D
:106510007D848C849B84AA84B984C884DF80EE80C7
:10652000FD800C811B81AA81B981CE0FD11D0FB6D0
:10653000F894DEBF0FBECDBFED010895AA1BBB1BB3
:1065400051E107C0AA1FBB1FA617B70710F0A61B73
:10655000B70B881F991F5A95A9F780959095BC0194
:10656000CD01089597FB072E16F4009406D077FD11
:1065700008D0E4DF07FC05D03EF4909581959F4F4D
:106580000895709561957F4F0895EE0FFF1F059058
:10659000F491E02D0994082E817006940694811DD3
:1065A0000694811D0694811D0694811D0694811D0B
:1065B0000694801D089569279627692778278727DD
:1065C000782708958F929F92AF92BF92CF92DF92D9
:1065D000EF92FF92CF93DF93EC01688179818A81FA
:1065E0009B81611571058105910521F464E279EDC6
:1065F0008BE597E02DE133EF41E050E0BFD049015A
:106600005A019B01AC01A7EAB1E4D4D06B017C0133
:10661000ACEEB4EFA5019401D9D0DC01CB018C0D17
:106620009D1DAE1DBF1DB7FF03C00197A109B04856
:1066300088839983AA83BB839F77DF91CF91FF9053
:10664000EF90DF90CF90BF90AF909F908F90089584
:10665000B9CF80E091E0B6CFA0E0B0E08093000138
:1066600090930101A0930201B09303010895FB01EF
:10667000DC0102C005900D9241505040D8F70895BA
:10668000FB01DC0104C08D910190801921F441507F
:106690005040C8F7881B990B0895FB01DC0102C02C
:1066A00001900D9241505040D8F70895DC0101C08F
:1066B0006D9341505040E0F70895DC01CB01FC019F
:1066C000F999FECF06C0F2BDE1BDF89A319600B44B
:1066D0000D9241505040B8F70895F999FECF92BD00
:1066E00081BDF89A992780B50895A8E1B0E042E00D
:1066F00050E0E5CFDC01A40FB51F4150504040F001
:10670000CB01840F951F2E9105D041505040D8F7F2
:106710000895262FF999FECF92BD81BDF89A019771
:1067200000B4021639F01FBA20BD0FB6F894FA9AD9
:10673000F99A0FBE08950396272FECDFEADF252F85
:10674000E9DF242FE7CF0196272FE4DFE2CFDC013A
:10675000CB0102C02D9105D041505040D8F708958B
:10676000262FF999FECF1FBA92BD81BD20BD0FB66D
:10677000F894FA9AF99A0FBE01960895052E97FBA0
:1067800016F400940FD057FD05D024D007FC02D09A
:1067900046F408C050954095309521953F4F4F4F96
:1067A0005F4F089590958095709561957F4F8F4FBD
:1067B0009F4F089531D0A59F900DB49F900DA49F39
:1067C000800D911D11240895B7FFF4CFF3DF821BD4
:1067D000930B0895A1E21A2EAA1BBB1BFD010DC04D
:1067E000AA1FBB1FEE1FFF1FA217B307E407F50781
:1067F00020F0A21BB30BE40BF50B661F771F881F5D
:10680000991F1A9469F760957095809590959B01F2
:10681000AC01BD01CF010895A29FB001B39FC0019B
:10682000A39F700D811D1124911DB29F700D811DBC
:106830001124911D0895F894FFCF180D1D0D1F0D03
:10684000240D340D340D340D340D340D340D340D50
:10685000340D260D2A0D2D0D320D420D480D4C0D17
:106860008A13B013B613B013B61308142914B61351
:106870002F153C15601A6B1A9F1AEB1A2D1B741BEF
:106880008A1B8D1B901B951B981B9D1BA01BA31B7C
:10689000A61BA91BAC1BAF1BB21BB51B511C211D9A
:1068A000261D291D361D3A1D451D481D531D561D0B
:1068B000611D641D6F1D83248624B1248B24B6249E
:1068C0009024BB249524C0249A24C524A824AE2453
:1068D00083248624B1248B24B6249024BB249524BD
:1068E000C0249A24C524172F322F392F102D102D94
:1068F0006C2F7C2F8F2FD02FD52F102D102D102DDA
:10690000DD2FFE2C022D352D422D4D2D582D5B2DCA
:10691000922DBD2DFB2C022FC02DC32DC62DF12D88
:106920002D2E302E322E662EE52FF32F0A30102D0D
:0A693000102D3F305C307F309830AE
:10693A000100000000FF00FFFF0300000100D40C6B
:10694A00FC11140E12121712F3110100FFFFDC0BD7
:10695A0071F924BD07B40044227B49012701AC0028
:10696A004F0268028802003131295A1B750A3033F6
:10697A00673666F6F5F4F1C69593929190949697D8
:10698A00343554535251504F4E4D4C4B4A49484757
:10699A00464544434241403F3E3D3C3B3A39383705
:1069AA00363534333231302F2E2D2C2B2A292827F5
:1069BA00262524232221201F1E1D1C1B1A191817E5
:1069CA00161514131211100F0E0D0C0B0A080C3C9D
:1069DA000C700CA40CD80CD83CA43C703C3C3C0871
:1069EA003CE040D040C040B040A040904080407061
:1069FA00406040504040403040204010400040E05D
:106A0A0030D030C030B030A030903080307030603C
:106A1A0030503040303030203010300030E020D05C
:106A2A0020C020B020A0209020802070206020501C
:106A3A002040203020202010200020E010D010C05C
:106A4A0010B010A0109010801070106010501040FC
:106A5A00103010201010100010E000D000C000B05C
:106A6A0000A00090008000700060005000400030DC
:106A7A0000200010000000020202020202020202CA
:106A8A0002040404040404040404040404040404BE
:106A9A0004040404040404040404040404040404AC
:106AAA00040404040404040404040404040404049C
:106ABA00040404040404040404040404040404048C
:106ACA000404040404040404040404040F3F7FBD02
:106ADA00E200E900EA00B500B600B700CD00830184
:106AEA00CC008A0192019401210223022402250288
:106AFA00260227022A02B300B4006F0070009F0129
:106B0A00CB019F02A002E200E900EA00B500B6004C
:106B1A00B700CD008301CC008A01920194012102C1
:106B2A00230224022502260227022A02B300B40005
:0C6B3A006F0070009F01CB019F02A002C1
:00000001FF
